:1000000086C30000BCC30000BAC30000B8C3000030
:10001000B6C30000B4C30000B2C30000B0C3000008
:10002000AEC30000ACC300000C9498310C94803235
:100030000C944D31A4C30000A2C30000A0C3000073
:100040009EC300009CC300009AC3000098C3000038
:100050000C94DB300C94743192C3000090C3000008
:100060008EC300008CC300008AC3000088C3000058
:1000700086C3000084C3000082C3000080C3000068
:100080007EC300007CC300007AC3000078C3000078
:1000900076C3000074C3000072C3000070C3000088
:1000A0006EC300006CC300006AC3000005010902B2
:1000B000A10185020901A1000509190129081500FE
:1000C0002501950875018102050109300931158165
:1000D000257F95027508810609381581257F9501D0
:1000E00075088106050C0A38021581257F95017572
:1000F000088106C0C005010980A101850319012AF4
:10010000B700150126B700950175108100C0050CD8
:100110000901A101850419012AA002150126A002E6
:10012000950175108100C00660FF0961A101096297
:10013000150026FF00952075088102096315002629
:10014000FF00952075089102C005010906A101056F
:100150000719E029E7150025019508750181029529
:1001600001750881010507190029FF150026FF0008
:100170009506750881000508190129051500250156
:10018000950575019102950175039101C00000006C
:10019000000000000000000000000000000000005F
:1001A000000000000000000000000000000000004F
:1001B000007E0F00D4FFFFFFC700000078000000A2
:1001C00000000000002A2B280000000000000000B2
:1001D000000000000000000029000000002C1E3478
:1001E00020212224342627252E362D3738271E1F7E
:1001F000202122232425263333362E37381F0405A9
:10020000060708090A0B0C0D0E0F10111213141516
:10021000161718191A1B1C1D2F3130232D350405F4
:10022000060708090A0B0C0D0E0F101112131415F6
:10023000161718191A1B1C1D2F3130354C09025B7B
:1002400000030100A0FA09040000010301010009F4
:100250002111010001224400070581030800010962
:100260000401000203000000092111010001222203
:100270000007058203200001070503032000010990
:100280000402000103000000092111010001227B8A
:10029000000705840320000112010002000000088D
:1002A000D44510010100010203011C03760069001E
:1002B00061006C003A0066003600340063003200D2
:1002C0006200330063000000120359004D00440037
:1002D0003200310020007600320000000A0359008D
:1002E0004D0044004B000000040309043A003B00A9
:1002F0003C003D0053005400550056005F00600074
:10030000610067005C005D005E00570059005A0004
:100310005B002C00215262006300580021780578B0
:1003200001000100010001000100010001000100C5
:1003300001000100010001000100010001000100B5
:1003400001000100010001000100010000000000A7
:100350000000000000000001010203040506080A75
:100360000C0F1114181C2024292E33393F464C53EE
:100370005B626A7179818A929AA2AAB2B9C1C8CF26
:10038000D5DCE1E7EBF0F4F7FAFCFDFEFFFEFDFC47
:10039000FAF7F4F0EBE7E1DCD5CFC8C1B9B2AAA215
:1003A0009A928A8179716A625B534C463F39332E47
:1003B0002924201C1814110F0C0A08060504030236
:1003C000010100000000000000000000222325269B
:1003D00028292A2C2D2F3032333536383A3B3D3EF2
:1003E0004042434547494A4C4E5051535557595A3C
:1003F0005C5E6062646668696B6D6F717375777956
:100400007B7D7F81838587898A8C8E909294969854
:100410009A9C9E9FA1A3A5A7A8AAACAEAFB1B3B466
:10042000B6B8B9BBBCBEBFC1C2C3C5C6C7C9CACBBB
:10043000CCCDCED0D1D2D2D3D4D5D6D7D7D8D9D986
:10044000DADADBDBDBDCDCDCDCDCDDDDDDDDDCDCEF
:10045000DCDCDCDBDBDBDADAD9D9D8D7D7D6D5D40C
:10046000D3D2D2D1D0CECDCCCBCAC9C7C6C5C3C2D8
:10047000C1BFBEBCBBB9B8B6B4B3B1AFAEACAAA82D
:10048000A7A5A3A19F9E9C9A98969492908E8C8AE1
:1004900089878583817F7D7B79777573716F6D6BBC
:1004A0006968666462605E5C5A5957555351504E94
:1004B0004C4A4947454342403E3D3B3A3836353346
:1004C00032302F2D2C2A292826252322FFAA7F55BA
:1004D00040000101010101010101010202020202C9
:1004E00002020202030303030303030304040404DC
:1004F00004040405050505050606060606070707A4
:10050000070708080808090909090A0A0A0B0B0B5A
:100510000C0C0C0D0D0D0E0E0E0F0F0F10101111F7
:10052000111212131314141515161617171818197B
:10053000191A1A1B1B1C1D1D1E1E1F2020212222E2
:10054000232424252626272829292A2B2C2D2D2E25
:100550002F30313232333435363738393A3B3C3D3F
:100560003E3F404142434445464748494A4C4D4E30
:100570004F50515354555658595A5B5D5E5F6162F6
:1005800064656668696B6C6D6F7072737577787A85
:100590007B7D7E8082838587888A8C8E8F919395E0
:1005A00096989A9C9EA0A2A3A5A7A9ABADAFB1B304
:1005B000B5B7BABCBEC0C2C4C6C9CBCDCFD1D4D6E4
:1005C000D8DBDDDFE2E4E7E9EBEEF0F3F5F8FAFD86
:1005D000FF1E0F0500047F3F1F643214643214783D
:1005E0003C1E1E140A05FD377A585A000004E6D650
:1005F000B4460200210116000000742FE5A3E001BB
:100600006E00E85D003D8889C65436C3174FE4E9A3
:10061000A5387CCE72B22DE3DE128598FEC4B78871
:100620009F4C500E9BDAC9249131703D7633D23401
:100630004FFB2B7ED9B56480AD741B467D5F868CE5
:100640000E8CDC8DF95D68A74AD311383C756C625D
:100650008BD89EBE64339D6C4B5810CE78A8F04367
:10066000DB5B63ED1E11B246D3D4DBFBB1DFD99E59
:10067000FC6AD655BF5676ABBAA4BAA3B696BEE30B
:10068000FEF9201F244680F8FE8D9E324894F4F334
:10069000F24E2B2C1837C0CA02F5FE027F6FAD6AEE
:1006A000276A6DFC051A3CB149ACAC62FEA1392841
:1006B000C84F7BD29DFBADD307F9F888CD73B61C2C
:1006C00032C74F2FBDDD27C61B3C975CAE3A6DC0CD
:1006D000FA4C460212B2F549FA04326A210074DA81
:1006E000F3F4E1760A9781766B5E5FC420009CD7B5
:1006F0006FC13911D3C900018402EF0200007354A5
:100700002CB1B1C467FB020000000004595A112447
:100710001FBECFEFDAE0DEBFCDBF04B603FE18C0C8
:100720008091A0049091A104A091A204B091A3048F
:100730008730904BA740B04B59F41092A004109210
:10074000A1041092A2041092A304E0E0F8E309953A
:1007500024E0AEEDB1E001C01D92A03AB207E1F78E
:1007600011E0A0E0B1E0E8EBFAE602C005900D92DE
:10077000AE3DB107D9F70E94BA280C94D53440CCCD
:100780009C01FB019A9581159F4120F5832F817073
:10079000B32FB270AA27732F74706627532F587027
:1007A000442734FF0DC08295807FAB2B09F0806217
:1007B000672B09F08064452B09F08068099508953E
:1007C000AB2B09F08260672B09F08460452BB1F3F5
:1007D0008860F4CF80E0F2CF80939C0408958093EA
:1007E0009D04089521E030E001C0220F8A95EAF7C8
:1007F00080919D04822BF3CF21E030E0A90102C05B
:10080000440F551F8A95E2F7CA01809590919D0487
:100810008923E5CF282F963090F5843080F534E099
:10082000939FC0011124820F911D282F277041E052
:1008300001C0440F2A95EAF723E0969587952A95FB
:10084000E1F7FC01EE0FFF1FE80FF91FED5CFC4F15
:1008500020E030E070E05191DF01CB01022E02C0B8
:10086000969587950A94E2F7817081958527842370
:1008700085278E932F5F3F4F2330310561F7089511
:10088000282F963078F5843068F534E0939FC001C6
:100890001124820F911D682F677023E0969587952C
:1008A0002A95E1F7FC01EE0FFF1FE80FF91FED5C41
:1008B000FC4F40E050E080E0219130E0062E02C085
:1008C000369527950A94E2F721703327042E01C04C
:1008D000220F0A94EAF7822B4F5F5F4F4330510596
:1008E00059F7089580E0089590919D0421E030E04B
:1008F000F90101C0EE0F8A95EAF7D90102C0AA0FEB
:10090000BB1F6A95E2F7EA2B01C0220F4A95EAF76E
:10091000892F8E23E81303C0892F822B60CF209567
:10092000822F8923FBCF8091E1029091E0029813FE
:1009300001C008958F5F8770FACF9091E80380958A
:1009400089238093E803282F2770211110C089176D
:1009500071F090919F0492FF0AC0869586958695C6
:100960004BDF1092E8031092EA031092E903089516
:100970009091E503982B9093E5030895982F909517
:100980008091E50389238093E50308958091E40332
:10099000811531F01092E4031092EC031092EB03F6
:1009A0000895803E9105D9F1C8F48133910509F489
:1009B00082C048F48932910509F472C08A329105E7
:1009C00009F480C0089589339105E9F082389105D2
:1009D000D1F08533910509F45EC00895843E9105F8
:1009E000D9F148F4823E910539F1833E910549F1F0
:1009F00081EE90E00895863E9105C9F1873E91050C
:100A000009F43EC0089520919E042370211164C012
:100A100020919F0423FF14C089E290E00895209163
:100A20009E0420FD45C030919F0430FF09C024FD85
:100A300024C083EE90E0089520919E0422FDF7CF1C
:100A4000089520919E0422FD44C030919F0430FD02
:100A500043C024FFF5CF11C020919F0421FFF0CFA8
:100A600080919E0484FD09C087EE90E00895209156
:100A70009E0423FFE5CF24FFF7CF80E090E00895A8
:100A800020919E0423FD2BC030919F0431FFE1CFC4
:100A900084EE90E0089520919E0425FFD1CFBCCF35
:100AA00020919E0425FD1EC020919F0423FFC8CFE6
:100AB00089E390E0089520919E0426FFC1CF8AE249
:100AC00090E0089520919E0426FFBACF81E390E044
:100AD000089582EE90E0089580EE90E0089586EE0D
:100AE00090E0089585E390E0089590919E0492FF30
:100AF00010C041E0282F2471243009F040E031E09B
:100B0000282F2871283009F030E0431711F02CE02D
:100B1000822793FF10C041E0282F2471243109F06F
:100B200040E031E0282F2871283109F030E04317E8
:100B300011F02CE0822730919F0430FF10C051E06B
:100B4000282F2171213009F050E041E0282F287131
:100B5000283009F040E0541711F029E0822731FFD6
:100B600010C041E0282F2171213109F040E031E02F
:100B7000282F2871283109F030E0431711F029E0BF
:100B8000822794FD877E08951F93CF93DF9309DF1B
:100B9000EC01811522E5920708F052C0811540E56D
:100BA000940708F0CDC0803E910520F58D3C91055D
:100BB00008F0A1C0883A910570F4853A910508F0D3
:100BC00097C081309105B9F10497813A910598F168
:100BD000C0E0D0E030C0885A91094B97C8F7C85A96
:100BE000D0E0CC0FDD1FCF58DE4F0990D881C02D4B
:100BF000D46421C0811550E49507B0F4C11580E29A
:100C0000D80708F0B3C0C83ED105A8F0CE019A9528
:100C100081159F41E8F68D2F68DF182FCE019927A7
:100C2000C0DEEC01D12B07C09927BBDECC27DF70DB
:100C3000C82BD92BD06ACE01DF91CF911F91089597
:100C4000803842E59407C8F5803652E5950708F0EC
:100C50005BC0C03482E5D807D0F4C03292E5D90732
:100C600008F04BC08C2F8695869520E2829FC001AC
:100C70001124C37021E030E0A90102C0440F551FC8
:100C8000CA95E2F7EA01C82BD92BDD68D4CF8C2FA7
:100C900086958695877050E2859FC0011124C370A8
:100CA00021E030E0A90102C0440F551FCA95E2F7C8
:100CB000EA01C82BD92BDC68BECF803C52E59507F2
:100CC00058F48F71C03AD245A0F590E0982F88274C
:100CD000EC01C46FD06AAFCF805C9245809708F07A
:100CE00077CFDC2FCC27CC27DF71C06FD06AA3CFA2
:100CF000A497D064A0CFD0659ECFCF71D0E0DC2F79
:100D0000CC27C16FD06A97CF86958695877020E2F1
:100D1000829FC0011124C37021E030E0A90102C00C
:100D2000440F551FCA95E2F7EA01C82BD92BDA68A0
:100D300082CFDBDEC82FD0E0DC2FCC27D0627BCF88
:100D40008F71D3DE93E0CC0FDD1F9A95E1F7CC27AE
:100D5000DF70282F30E084FF05C050E1859F9001AF
:100D600011243327C22BD32BD06965CF8D2F8F71E0
:100D7000BCDE182FCE01992714DEEC01D12BDECF7B
:100D800080E00895F894E82FE295EF70F0E041A13B
:100D90008F7021E030E0B90102C0660F771F8A959D
:100DA000E2F7CB01962F9095942391A392A1892BE2
:100DB00082A3789408950895CF92DF92EF92FF92E4
:100DC0001F93CF93DF93172FE82FF0E0EF52FB4FE5
:100DD00071110CC0E4918E2F7E2F6E2FDF91CF9179
:100DE0001F91FF90EF90DF90CF900895E62EF12CA9
:100DF000C72ED12CF491EF2F86E0689F900111242B
:100E0000CFEFD0E0C901BE010E94E632AB01EE0C8B
:100E1000FF1C65E5649FC001659F900D1124E81AD1
:100E2000F90A6E2D660F6E0D7E01EC18FD08FE9D11
:100E3000D001FF9DB00D11248B2F169F700111243E
:100E4000EF2CFF246E01CE18DF087601FE9D6001B5
:100E5000FF9DD00C11247E01E61AF108B701169F00
:100E60007001179FF00C1124EF2CFF24CE19DF091D
:100E7000FC9F7001FD9FF00C11247F2D4330510524
:100E8000C1F02C3F334058F441305105B1F04230AD
:100E9000510509F0A2CFEB2F8F2D7F2F9ECF44302D
:100EA000510571F04630510509F497CF7B2F8D2DF8
:100EB00094CF7D2DEB2F8F2F90CF7F2FED2D8DCFCA
:100EC000EF2D7B2FF8CFCF93982F762F842FC22F23
:100ED000692F72DF472F282F8C2F90E0F9D2CF9106
:100EE00008958091DC03843060F483708460809383
:100EF000DC038091DF03853B18F084EB8093DF03F4
:100F000008958C3AB0F38370886AF1CFCF93DF9362
:100F10008091DC0380FD0BC0C0E0D0E020E040E029
:100F200060E0CE01D5D22196C830D105B9F79FD661
:100F3000DF91CF910895FF920F931F93CF93DF938B
:100F4000182F062FF42E8091DC0380FF0CC0C0E028
:100F5000D0E02F2D402F612FCE01BAD22196C8307C
:100F6000D105B9F7D3DFCDB7DEB7E5E00C944F3349
:100F7000CF93DF93EC012091DF039C81892F817057
:100F800090FD822F692F627091FD622F492F44706E
:100F900092FD422FD0DF8C8190E0019687709927D7
:100FA0008C83DF91CF910895982F762F842F2091F5
:100FB000DC0320FF0AC0453B08F084EB692FFCDE10
:100FC000962F672F482F892FB6CF0895CF93DF93A1
:100FD000EC01ECEDF3E0438162818C81E5DF8C81F3
:100FE0008F5F8C83DF91CF910895CF93DF93EC01D6
:100FF000EC81F0E0E453FC4F4491ECEDF3E06281CE
:101000008181D2DF8C818F5F8C83DF91CF910895B6
:10101000FF920F931F93CF93DF93EC01F12C00E02D
:1010200010E04091DF03453B08F044EB8C819801D0
:101030006091DE038F0D47DF0F5F1F4F8FE1F80ECA
:101040000830110571F762DF8C819A8190FF07C02B
:101050008F5F8C83CDB7DEB7E5E00C944F338150C2
:10106000F8CFEF92FF920F931F93CF93DF93FC0182
:101070008281FF24F39480FF02C0FF24FA94C0E031
:10108000D0E020E040E060E0CE0122D204E010E0B9
:10109000E12C8091A2028E0D89308CF18770082E90
:1010A000001C00088C170D0691F44091DF03040327
:1010B000A00111245595479555954795453B08F056
:1010C00044EB9E016091DE038091DD03FCDEEF0CBA
:1010D00001501040F1F62196C830D10591F616DF87
:1010E0008091A202F1E0FF120EC0811579F08150CB
:1010F0008093A202CDB7DEB7E6E00C944E3387FFB3
:10110000CECF885FCCCF8F5F8770F2CF87E0F0CFF4
:10111000CF93DF93C0E0D0E020E040E060E0CE017C
:10112000D7D12196C830D105B9F7C0E0D0E0809181
:10113000A102082E001C0008C817D00574F1809188
:101140000701082E001C00088C170D0634F1409191
:10115000DF03453B08F044EB9E016091DE03809184
:10116000DD03B1DE2196C830D10509F7CFDE8091CD
:1011700006019091A102980F9093A102209107017E
:10118000280F20930701121614F497301CF0819554
:1011900080930601DF91CF91089520E040E060E068
:1011A000CE0196D1DFCFA6E0B0E0E9EDF8E00C94F7
:1011B00030338D839E83AD81BE811496FC912F2F99
:1011C00030E0D9010E94C6349B01AC010E949434E6
:1011D0006B017C0180E290E09C012F1B3109F90139
:1011E000A5E5B0E0A70196010E94943469837A8353
:1011F0008B839C839F01DF010E941A339B010E9415
:1012000020339B01AC012C0D3D1D4E1D5F1D6981DE
:101210007A818B819C810E94A434022F30E00A32B3
:10122000B8F5C901880F991F820F931F959587956F
:10123000182F1095E12CF12C85E5D82ED01A8D2D84
:10124000E1FC802F412F153B08F044EB97016091A2
:10125000DE0339DE5FEFE51AF50A88E0E816F104EF
:1012600071F754DEAD81BE8114969C9181E0911599
:1012700019F0903219F48FEF8093050180910501E8
:10128000890FED81FE8184832696E8E00C944C332F
:1012900085E590E0AC01421B530B9A01CA01880F0F
:1012A000991F820F931F97FFC1CF0196BFCF0F9356
:1012B0001F93CF93DF93EC0120E030E06091DE03D9
:1012C0008091DD039C8189010F5F1F4F2430310520
:1012D00054F4911501F14091DF03453B08F044EBD4
:1012E000F2DD9801EBCF911116C04091DF03453B31
:1012F00008F044EBE8DD980108301105F9F606DE48
:101300008C8190E00196817099278C83DF91CF9139
:101310001F910F91089540E0EDCFA0E0B0E0E3E928
:10132000F9E00C942C338C01809186009091870019
:101330006CE070E00E94E6326017710768F0C80147
:1013400069E070E00E94E632262F972F822FCDB7FA
:10135000DEB7ECE00C9448338091860090918700D2
:10136000E0908600F0908700C0908600D0908700C3
:10137000C6E0D0E0BE010E94E63220E030E0060F79
:10138000171F211D311D4801590185E0880C991C4A
:10139000AA1CBB1C8A95D1F7C701BE010E94E63288
:1013A000E12CF12CA7019601260F371F411D511D7D
:1013B000C501B4010E94A43469017A01E09186005C
:1013C000F0918700CA01B9010E94CB329B01AC01A8
:1013D000DF010E9494349B01AC01C701B6010E9459
:1013E000CB32DC01CB012FE0B695A7959795879579
:1013F0002A95D1F720918600309187002817390768
:101400001A061B0620F48091860090918700282FF1
:101410009DCF8430E0F481111BC090918000977FB4
:10142000909380002091860030918700A82FB0E033
:101430000E94C63423E030E040E050E00E94A43433
:10144000C9016BDF90938D0080938C00089583E039
:10145000909180009860E4CF982F990F990F990F81
:1014600020914F032770922B90934F0321E09830E7
:1014700008F420E090914F0320FB90F990934F03E4
:10148000C8CF81152CE7920741F42091CD0230910D
:10149000CE02232B11F480E090E00895E4E5F3E020
:1014A00080E090E060E876E243EA56E225E137E248
:1014B000778366835187408733872287978786871C
:1014C000019670968830910599F708956A9A089563
:1014D000FC01EE0FFF1FE80FF91FE75FFD4F61836F
:1014E00040832283089510922E0410922D04EDEE75
:1014F000F3E08581811102C014821682379684E060
:10150000E532F807B1F70895AC01309130046091ED
:101510002F04232F621301C00895822F90E0FC0155
:10152000EE0FFF1FEB5DFB4F0190F081E02DE41704
:10153000F50791F467E0649FF001659FF00D1124B9
:10154000E351FC4F41E044832313E6CF01968370BF
:1015500099278093300408950196282F2370DACFBD
:10156000282F35EB2303C001112497FF04C08058B6
:101570009109892F089580589F4FFBCF80913E039A
:1015800080FD14C081FD14C082FD16C080913D0312
:10159000811581F08E3180F420E5829FC0011124F5
:1015A0006EE170E00E94FA32862F089584E108957A
:1015B00088E2089588E0089580E5089580913E03CB
:1015C00080FD17C081FD17C082FD19C080913C03CA
:1015D000811599F0883298F428E0829FC001112487
:1015E00068E270E00E94FA326115710551F0862FB1
:1015F000089562E0FCCF64E0FACF61E0F8CF68E0E4
:10160000F6CF81E00895FA01309709F00995089521
:10161000E091D602F091D702309739F00190F08135
:10162000E02D309711F00995089580E00895A3E02A
:10163000B0E0EDE1FBE00C9436339C0180910602B2
:101640009091070282179307B1F03093070220931D
:101650000602E091D602F091D702309761F0008443
:10166000F185E02D309739F083E089833B832A832D
:10167000CE01019609952396E2E00C945233A3E043
:10168000B0E0E5E4FBE00C9436339C018091040269
:101690009091050282179307B1F0309305022093D1
:1016A0000402E091D602F091D702309761F00084F5
:1016B000F185E02D309739F084E089833B832A83DC
:1016C000CE01019609952396E2E00C9452339C01D9
:1016D000FC0132968FEF90E04191461751F08F3F19
:1016E00019F4411101C0892F9F5F9630A9F78F3FF0
:1016F00009F40895280F311D87FD3A95F901628399
:1017000008959C01FC013296285F3F4F819186131A
:1017100002C0DF011E92E217F307C1F7089580911E
:10172000140108952FB7F89480910002909101025E
:10173000A0910202B09103022FBF0895962F20912D
:101740009F0422FF0EC0682F660F660F660F692B7D
:101750006093E80347D8E6DF9093EA038093E903B8
:10176000089540C89091E403292F2823211559F0AA
:10177000809589238093E403811531F0D3DF809332
:10178000EB039093EC03089580E090E0F8CFCADF7C
:101790002091410330914203232B211521F08093A6
:1017A000C0029093C1022091430330914403232B44
:1017B000211521F08093BE029093BF02E091D602E2
:1017C000F091D702309759F00680F781E02D3097DD
:1017D00031F082E080933F038FE393E00995089511
:1017E000611509F441C0E3E3E80FE33148F4F0E0A8
:1017F000E952FB4C0C940D33C1DE8195809342037A
:10180000C6CFBCDEFBCFBADE819580934103F8CF13
:10181000B5DEFBCFD3DE80934303F2CFCFDE8195DD
:10182000FACFCCDE819580934403EACFC7DEFBCFAD
:10183000815D990B21E030E001C0220F8A95EAF723
:1018400080914003822B80934003DACF80913E0346
:10185000816080933E03D4CF80913E038260F9CFB4
:1018600080913E038460F5CF409141038D3C59F453
:101870008091420387FF0DC010924203411559F435
:1018800010923D0308C08E3C81F4809142031816EB
:101890009CF3411581F08091430390914403892B7F
:1018A0008111AECF10923C03ABCF8F3C41F447FF88
:1018B000F0CF10924103809142038115E0CF803D2B
:1018C00019F41416B4F3E5CF90914303893D29F43C
:1018D0001916FCF610924303DCCF8A3D19F497FFEA
:1018E000D8CFF8CF909144038B3D29F497FFD1CF07
:1018F00010924403CECF8C3D19F41916CCF3C9CF06
:101900009FE2980F983090F4815D990B21E030E0D0
:10191000B90102C0660F771F8A95E2F7CB01809567
:1019200090914003892380934003B3CF8D3D31F4E0
:1019300080913E038E7F80933E03ABCF8E3D21F49A
:1019400080913E038D7FF7CF8F3D09F0A2CF80912C
:101950003E038B7FF0CF2FB7F89460910002709117
:10196000010280910202909103022FBF0895089511
:10197000FC019B018091F6019091F7018617970772
:1019800040F0672B29F48091E8008E778093E8007F
:10199000C90140E0009741F4411106C08091E80080
:1019A00082FF2FC080E008952091CF022115A9F178
:1019B0002530A9F12091E80023FD2DC02091E800F9
:1019C00022FDECCF2091E80020FFE4CF3091F3001E
:1019D0002091F200009719F02830310558F041E0CD
:1019E0002830310509F040E02091E8002E7720935F
:1019F000E800D0CF41914093F10001972F5F3F4F16
:101A0000E9CF8091CF02811541F0853041F080917E
:101A1000E80083FFC3CF81E0089582E0089583E06A
:101A200008958091F00187FF13C08091E80082FF44
:101A300006C08091E8008B778093E800089580913C
:101A4000CF028111F2CF08958091CF028115D9F391
:101A50008091E80080FFF8CF8091E8008E77ECCF8E
:101A60002091E4003091E50095E6A9012091EC0079
:101A7000822F817020FF06C08091E80080FF06C0A1
:101A800080E008952091E80022FD1AC08091CF02E5
:101A9000811589F0853089F08091EB0085FD0FC0BC
:101AA0002091E4003091E50042175307F9F29A952E
:101AB000E1F684E0089582E0089583E0089581E0EE
:101AC0000895E8EDF0E080818E7F80831092E2003F
:101AD0001092DA001092E100A0EEB0E08C918160EB
:101AE0008C9380818F77808319BCA7EDB0E08C91B7
:101AF0008E7F8C9380818F7E80831092EF0108957A
:101B0000E091D602F091D702309739F00284F38544
:101B1000E02D309711F060E209950895982F909389
:101B2000E900891771F07091EC002091ED0050915F
:101B3000F00021FD09C09F5F973089F78093E9008D
:101B40000895762F242F50E03091EB003E7F3093A4
:101B5000EB003091ED003D7F3093ED003091EB00D4
:101B600031603093EB007093EC002093ED005093C4
:101B7000F0002091EE0027FDDECF0895A0E0B0E058
:101B8000E4ECFDE00C943033C8EDD0E088818F7E2A
:101B90008883E7EDF0E080818160808384E082BF0C
:101BA00081E08093EF0188818E7F888302EE10E0D0
:101BB000F80110821092DA0081EEC82ED12CF601C5
:101BC000108288818F778883888180688883888164
:101BD0008F7D888319BC1092CF021092EE01109273
:101BE000B0021092ED0190EEE92EF12CF701808108
:101BF0008B7F808388818160888342E060E080E021
:101C00008DDFF60180818E7F8083F8018081816085
:101C10008083808188608083F70180818E7F8083CC
:101C2000888180618883CDB7DEB7E8E00C944C33BF
:101C3000E091E1029091E00229E0E91302C080E026
:101C40000895AE2FB0E02E9FF0011124EE51FD4F0C
:101C50003181361306C03081381303C03581341307
:101C600004C0FD013196E770E8CF81E008953EB1F0
:101C70003B7F2EB124604FB7F89489E092E0FC01DD
:101C80000196508168E02EB9000000C057FF3EB9B0
:101C9000550F000000C000C000C03EB900C06A95EA
:101CA00091F752E08132950751F74FBF8FE594E0ED
:101CB0000197F1F700C00000089581E08093E000F3
:101CC00080E28093D8001092C9008FE19EE40197D2
:101CD000F1F700C0000087E090EBDC018093A004E6
:101CE0009093A104A093A204B093A30488E19CE084
:101CF0000FB6F894A895809360000FBE9093600093
:101D0000FFCF0F931F93CF93DF938B01EA01909145
:101D1000CF02943051F58093E9008FEF9091E80065
:101D200095FD06C095ED9A95F1F700008A95B1F7FB
:101D30008091E80085FF19C093DE811111C0809168
:101D4000E80085FD06C08091E8008E778093E8006A
:101D5000F3CFF80181918F018093F100219779F7FA
:101D60008091E8008E778093E800DF91CF911F91FA
:101D70000F910895792F603229F440E250E0682FE6
:101D800082E0BFCF0895CF93DF93D82FC92F48E0CB
:101D900050E0682F792F81E0B4DF88E0ED2FFC2F31
:101DA000A8EFB1E001900D928A95E1F7DF91CF9114
:101DB0000895BC0146E050E084E0A3CFBC0143E0BD
:101DC00050E084E09ECF90919F0492FB222720F95F
:101DD000281779F080FB92F990939F0460919E04FC
:101DE00070919F0484E090E00E945D3482E00C9446
:101DF0009D040895FC01608186E090E00C944334DA
:101E000080914F0381FD11C0826080934F038FE466
:101E100093E0F0DF1092AB021092AA021092A90296
:101E200080916F00816080936F00089580914F03CF
:101E300081FF11C08D7F80934F038FE493E0DADF41
:101E400080916F008E7F80936F0080914F03869505
:101E500086958695DECA08951F93CF93DF93C62F8C
:101E6000122F632F982F942B9430C0F4C630B0F407
:101E700098E0C99FE0011124C40FD11DC40FD11DEA
:101E800090E3899FC00DD11D1124CE0189960E9437
:101E90004334612FCE018A960E944334DF91CF9163
:101EA0001F910895CF93DF93C091E5038091E703DD
:101EB000C82B8091E4038115F1F034DC2091EB0311
:101EC0003091EC03821B930B8838934110F00E94F1
:101ED000C604D091E40320E082EE91E0FC01308161
:101EE000019631112F5F31E0883E9307B9F7211138
:101EF0000E94C604CD2BC093E00148E050E068ED9D
:101F000072E080EE91E00E94FE33892BB9F088E008
:101F1000E0EEF1E0A8EDB2E001900D928A95E1F7D4
:101F2000E091D602F091D702309741F00280F38120
:101F3000E02D309719F080EE91E00995DF91CF9177
:101F40000895CF931092E503C6E0E2EEF1E0DF01E1
:101F50008C2F1D928A95E9F780E090E068DB80E0A5
:101F600090E08DDB1092E7039DDFEFE3F3E0DF010C
:101F70001D92CA95E9F710923D0310923C0310920E
:101F80003E0305DCCF910895DCDF2FEF84E39CE076
:101F9000215080409040E1F700C0000088E19CE0C3
:101FA0000FB6F894A895809360000FBE90936000E0
:101FB000FFCFAAE2B0E0EFEDFFE00C94353380EF05
:101FC00091E0FC0101962091F100208321E0883FFF
:101FD0009207B9F78091F101893009F457C0C8F42C
:101FE000823009F4B2C0833009F482C0813081F1BB
:101FF0008091E80083FFE6C08091F0019091F101AB
:102000009A3008F0DFC0E92FF0E0E651FB4C0C9469
:102010000D338A3009F489C08B3051F78091F0017B
:10202000813231F78091F4019091F501892B01F70C
:102030008091E800877F8093E800F3DC81E0909155
:10204000F201911101C080E0809315017ADFD0CFB9
:102050008091F001813A61F68091E800877F80935A
:10206000E8008091F4019091F501892B59F060E02E
:1020700080E090E070E07CDC8091E8008B778093DA
:10208000E800B6CF68E088EF91E0F4CF8091F001EE
:10209000813209F0ADCF8091F4019091F5018D7FEF
:1020A000892B09F0A5CF8091E800877F8093E80015
:1020B0008091E80082FF17C09091F3008091F200B8
:1020C000029731F48091F100813011F0863021F4D3
:1020D0008091F100809314018091E8008B778093C8
:1020E000E8009FDC85CF8091CF028111E1CF80CFC6
:1020F0008091F001813A09F07BCF8091F4019091B9
:10210000F501892B09F074CF8091E800877F8093D7
:10211000E8008091E80080FFFCCF8091150180935A
:10212000F1008091E8008E77DACF8091F001813262
:1021300009F05ECF8091E800877F8093E80071DC32
:102140008091F3018093130153CF8091F001813A84
:1021500009F04ECF8091E800877F8093E80080915E
:10216000E80080FFFCCF80911301D9CF803889F03F
:10217000823841F58091F4018F70873018F5809393
:10218000E9008091EB0085FB882780F91092E90037
:1021900006C08091B002880F9091ED01892B90913B
:1021A000E800977F9093E8008093F1001092F1008F
:1021B0008091E8008E7723C0811116C08091F201D2
:1021C000813009F18091E80083FF0AC08091E80026
:1021D000877F8093E8008091EB0080628093EB0022
:1021E000AA96E3E00C945133823061F78091F201BA
:1021F000811581F01092E9008091E800877F80933B
:10220000E8000FDCDFCF81E0933009F080E08093BD
:10221000B002F0CF8091F4018F702FEF280F26309D
:1022200088F68093E9002091EB0020FFE3CF933004
:1022300031F48091EB0080628093EB00DBCF9091D2
:10224000EB0090619093EB0021E030E0A90102C027
:10225000440F551F8A95E2F74093EA001092EA0076
:102260008091EB008860E8CF8111ACCF1091F20132
:102270001F778091E3008078812B8093E300809129
:10228000E800877F8093E800CCDB8091E80080FF46
:10229000FCCF8091E30080688093E30083E011111C
:1022A00001C082E08093CF028DCF8058823008F049
:1022B00089CF8091F2019091F3018C3D53E0950715
:1022C00091F583E08A838AE289834FB7F894DE012F
:1022D000139620E03EE051E2E32FF0E050935700E8
:1022E000849120FF03C082958F703F5F8F708A308A
:1022F000C0F0895C90E08D939D932F5F243161F74E
:102300004FBF8091E800877F8093E8006AE270E029
:10231000CE0101962DDB8091E8008B778093E80059
:1023200051CF805DE7CF292F33272330310509F4C2
:102330004EC078F52130310509F488C08BE590E076
:10234000EDE3F2E02230310509F03CCF2091E800C6
:10235000277F2093E8002091F6013091F701821742
:10236000930708F49C0140E02115310509F073C082
:10237000411171C08091E80082FDCDCF8091CF02E4
:10238000811549F2853039F28091E80083FFF2CF60
:10239000C2CF8091F4019091F5012132310509F409
:1023A00046C02232310509F00DCF8330910508F087
:1023B00009CFFC01EE0FFF1FE05DFE4F0190F081A1
:1023C000E02D835D9E4FDC018C9190E010C09C015C
:1023D0003327823021F12330310568F4232BB9F4FF
:1023E000E8EEF2E0E4918E2F90E0E8EEF2E0009764
:1023F00009F4E8CEABCF2330310509F0E3CEEAEAA9
:10240000F2E0E4918E2F90E0EAEAF2E0F0CFECED1A
:10241000F2E0E4918E2F90E0ECEDF2E0E8CFE8EC12
:10242000F2E0E4918E2F90E0E8ECF2E0E0CF833030
:10243000910508F0C7CEFC01EE0FFF1FEA5CFE4FCE
:102440000190F081E02D89E090E080CF82E190E082
:10245000E8E9F2E07BCF8091CF02811509F45BCFF0
:10246000853009F458CF8091E80083FD54CF8091E6
:10247000E80082FD7FCF8091E80080FF75CF9091CA
:10248000F3008091F2002115310519F08830910593
:1024900050F041E0089709F040E08091E8008E7725
:1024A0008093E80061CF44914093F1003196215030
:1024B00031090196E8CF803809F084CE8091E80098
:1024C000877F8093E8008091EE018093F10070CEC9
:1024D000811178CE1091F201123008F073CE809104
:1024E000E800877F8093E8001093EE019ADA1115D7
:1024F000D9F084E08093CF0242E061EC81E00EDB12
:1025000042E261EC84E00ADB42E261EC82E006DB5D
:1025100042E260EC83E002DB8091CF02843051F430
:1025200082E0809316014ECE8091E30087FDE1CFDB
:1025300081E0E0CF81E0F5CFCF93C82F811599F0EE
:102540008CEF8C0F813A88F4E2EEF1E088EE91E0B6
:102550002191C217B1F18E179F07D1F76C2F80EE32
:1025600091E0B5D89FDCCF91089580E28C0F883040
:1025700048F4C77081E001C0880FCA95EAF70E944D
:10258000B804F0CF8BE58C0F833030F42C2F24521D
:10259000330BC9014CD8E7CFE8E5EC0FEB3148F439
:1025A000F0E0EE0FFF1FE955FE4F8081918167D863
:1025B000DACF83E38C0F8331B0F661E08C2F10D932
:1025C000D2CF6C2F80EE91E09CD86CDCC7CF811508
:1025D00059F19CEF980F913A28F4682F80EE91E022
:1025E00090D860CC90E2980F983050F4877091E0CA
:1025F00001C0990F8A95EAF7892F0E94BE04F1CF96
:102600009BE5980F933018F480E090E010C898E5AF
:10261000980F9B3118F480E090E031C893E3980F55
:10262000933110F460E0DCC808951F93CF93DF93DB
:10263000182FEB0181DF209731F4812FC8DFDF9164
:10264000CF911F9108958FE99FE00197F1F700C0A6
:1026500000002197F0CF811519F00E94B80422CC18
:102660000895811519F00E94BE041CCC08958115AF
:1026700031F09091E703892B8093E70313CC089501
:10268000811539F080959091E70389238093E703C2
:1026900009CC089580915003811521F082E2F0DF8A
:1026A000109250030895CF93DF93EC014A855B8528
:1026B0006E857F850E94030B9B8190958091E70337
:1026C00089238093E7038C810E94BE04EBDB86E0C4
:1026D000FE0111928A95E9F7DF91CF910895CF938A
:1026E000DF93EC018D8181FD13C082608D83809129
:1026F000E7039B81892B8093E7038C810E94B804B8
:10270000D1DB488559856E857F85CE010E94030BFC
:102710001092D5031092D4038D8180FD02C0CE01AA
:10272000C2DFDF91CF91089586E090E00E942234CD
:1027300080934F0382FD06C08DE180934F038FE4A9
:1027400093E058DB80914F03803220F087708861DE
:1027500080934F0390914F03892F817090FF04C0A5
:10276000892F8695869586950C94090A0F931F9359
:10277000CF93DF93982F942B943018F5663008F59B
:1027800028E0629FE0011124C40FD11DC40FD11DA8
:1027900030E3839FC00DD11D1124CE0189960E9484
:1027A0002234082F10E0102F0027CE018A960E94B5
:1027B00022349801282BC901DF91CF911F910F91ED
:1027C000089580E090E0F8CF462F672F2091D20245
:1027D0003091D302232B81F4703F39F4403F61F4F0
:1027E0008091D0029091D1020895763028F4982FEC
:1027F000942B943008F4BACF80E090E00895A0E0E4
:10280000B0E0E5E0F4E10C9431337C0100919D04EB
:1028100080919C04082BC3E0D0E010E0C8010C2E8E
:1028200002C0959587950A94E2F780FD09C021972B
:10283000A8F7D12C8D2DCDB7DEB7E7E00C944D3342
:10284000DC2EB7018C2FC0DF0E94C405019779F3FD
:10285000F1CF0F931F93CF93FC0187819085009751
:1028600089F4858100811181811581F0611571F0F4
:10287000C801C5DFC82F682FC8010E940A04B8012B
:102880008C2FA2DFCF911F910F910895C8010E9454
:102890004004C82FF4CFCF93DF93D82FC92FAFDFD9
:1028A0006D2F7C2F91DF0E94C405DF91CF91089599
:1028B000FC0184818115B1F0878190850097A1F09A
:1028C0000E94C405282F92959F709630B9F080F42D
:1028D000925F9F70923030F4203FD1F058F481E045
:1028E000283E58F080E0089580819181D4DFEACFBE
:1028F0009A5FEFCF81E0243FA9F7089591E0813FEF
:1029000009F090E081E0283E08F080E0892B0895EE
:1029100081E00895382F292FCB01A32FB22F8737BD
:1029200022E09207A105B10520F487579E4F0C9431
:10293000223480E0089585E290E00E9422348B30BA
:1029400089F486E290E00E9422348B3459F487E2C5
:1029500090E00E94223491E0823609F090E0892FC5
:102960008170089580E0FCCFA0E0B0E0EAEBF4E1F4
:102970000C942F33EC018881811509F1813009F025
:1029800045C08981813051F48A81239660E570E0E9
:10299000893311F060E070E048DEEDCF823021F441
:1029A0008A812396C9DDE7CF833021F48A8123967B
:1029B0000EDEE1CF843041F022968111DCCFCDB71D
:1029C000DEB7E9E00C944B338A81239620E030E0B7
:1029D0009AE0682F6053770BAB016A30710560F0A5
:1029E0002115310551F3EFE9FFE03197F1F700C010
:1029F000000021503109F4CF929FB001939F700DD8
:102A000011249A01260F371F8991E3CFE82FF0E0B8
:102A1000E354FE4FB490282F26952695269530E056
:102A2000F901E355FE4FE4908770F12C082E02C0A7
:102A3000F594E7940A94E2F7E0FAEE24FF24E0F834
:102A4000F901E356FE4FC490D12C082E02C0D59454
:102A5000C7940A94E2F7C0FACC24DD24C0F8F90147
:102A6000E357FE4F049110E002C0159507958A9533
:102A7000E2F701701127E114F10411F081EE5CDD41
:102A8000C114D10411F086EE57DD60E070E08B2DAB
:102A9000CCDDC114D10411F086EE99DDE114F1040E
:102AA00011F081EE94DD0115110521F060E070E078
:102AB0008CE2BBDD21965FCFAAE0B0E0E2E6F5E173
:102AC0000C942B33C090CD02D090CE0281E090E0E8
:102AD0009093CE028093CD02812C912C10E0540172
:102AE00000E019C021E030E0123020F4F7018591B8
:102AF00095919C01472D602F812FAED9739422E0D0
:102B0000E20EF11C34E07312EDCF0F5F84E0A80EEB
:102B1000B11C063049F0C501880F991FFC01E45132
:102B2000FD4F7F01712CDECF1F5FF8E18F0E911CEE
:102B30001430A9F61A8219821C821B821E821D8201
:102B400018861F8288EC90E09A87898709EE10E04A
:102B50009E012F5F3F4F79014AE050E0B801C70165
:102B60000E946134065F1F4F5701093331E013079C
:102B700099F78AE0F70111928A95E9F74AE050E067
:102B8000B801C5010E946134065F1F4F0938F1E0AA
:102B90001F07A1F7D092CE02C092CD022A96EDE097
:102BA0000C944733AAE0B0E0E8EDF5E10C94303343
:102BB000E1E2F2E080E5DF011D928A95E9F7EDEEB2
:102BC000F3E088E3DF011D928A95E9F781E2C82EE0
:102BD00082E0D82E7F0109E311E0F701D182C082A3
:102BE0004AE050E0B801CE0101960E94123488E01C
:102BF000FE013196D60101900D928A95E1F7898503
:102C00009A85D70113969C938E931297BAE0CB0EB8
:102C1000D11CE7E0EE0EF11C065F1F4F0938F1E012
:102C20001F07D9F62A96E8E00C944C33282FCB01E5
:102C3000283070F44AE0249F90011124B9016751B3
:102C40007F4F4AE050E00E94123480E090E0089507
:102C50008FEF9FEF0895AAE0B0E0E1E3F6E10C9476
:102C600036339C0197558115914068F4BE016F5F22
:102C70007F4F822FDBDF892B31F489859A852A9655
:102C8000E2E00C94523388EC90E0F9CFA0E0B0E0A1
:102C9000ECE4F6E10C943133162FD72FC42FD22E4B
:102CA0008115A1F04093D8030E94920B9093EC0100
:102CB0008093EB01C77081E001C0880FCA95EAF7E5
:102CC000CADCCDB7DEB7E7E00C944D339091D80362
:102CD000491335C0E090EB01F090EC010E94920B9B
:102CE0009C012E193F097901812F9D2FB4DFE81631
:102CF000F90628F5D0E2DD0DCD1591F0C77011E091
:102D0000812F01C0880FCA95EAF7ABDCD83040F4B8
:102D10008D2D877001C0110F8A95EAF7812F9BDCFA
:102D200060E070E0802F81DCD83058F62D2D2770C0
:102D300081E001C0880F2A95EAF793DCC2CFC77003
:102D400081E001C0880FCA95EAF7F7CFA0E0B0E0B4
:102D5000ECEAF6E10C942A33FC018280648081E085
:102D60008483ECECF3E09490EBE4F4E0E4910091E4
:102D7000DF030695015810E0000F111F012F1127E6
:102D8000C9E7D2E0C12CD12CAA24AA94B12C772473
:102D90007A94E919EE2EF12C83E0881630F48091B4
:102DA000DD0388838091DE03898361101AC01B8252
:102DB0001A824A81453B08F044EB9601698188817B
:102DC0000E9463078FEFC81AD80A259688E0C816B4
:102DD000D10411F70E948607CDB7DEB7EEE00C9460
:102DE00046338B818115E9F081508B83789EC00139
:102DF00011246C8170E00E94E632FB01FF27E4534E
:102E0000FC4F8491E82FE9197E9EC0011124B7017F
:102E10000E94E6328091DF03689FB00111247A831B
:102E2000C8CF0E94DA33B5010E94FA3280179107A9
:102E30000CF0BFCF83E0881688F00E94DA33B5012A
:102E40000E94FA3288830E94DA332091DE032695AD
:102E5000622F70E00E94FA32280F29831A82809133
:102E6000DF03893C20F088EC8C838B83A2CF8431F4
:102E7000D8F784E1F9CF0F93CF93DF93CCEDD3E074
:102E8000488159816A817B8188E090E00E945534B5
:102E9000288139814A815B816C817D818E819F810E
:102EA00000E20E947833622F83E290E00E94433474
:102EB000DF91CF910F910895ECEDF3E085E08083F1
:102EC00011828FEF828384EB83831482CF01D3CF6F
:102ED0008091E003833018F48F5F8093E0038CEDE2
:102EE00093E0C9CF8091E003811519F08150809360
:102EF000E0038CED93E0BFCFA0E0B0E0E2E8F7E1C3
:102F00000C942D33082FF62E142FE22E9091DC0313
:102F100090FF26C0E92FE695E695AE2FB0E0A45CC1
:102F2000BE4F8C918093DA039C7F9430F1F4842F10
:102F3000453B08F084EB602F7F2D0E94DC06962F26
:102F4000672F482F892F0E949B070093DD03F09283
:102F5000DE031093DF03E11419F08CED93E08BDFB7
:102F6000CDB7DEB7EBE00C944933823019F4109101
:102F7000DF03EBCF863019F40091DD03E6CF893013
:102F8000D9F3893111F7E9512E2F2170922EE69550
:102F9000F0E0E453FB4FE491CE2FD0E0A12CB12C14
:102FA000C12CD12CC50123E0969587952A95E1F790
:102FB000911015C0800F412F153B08F044EB96018E
:102FC0006F2D0E9463078FEFC81AD80AAC0EBD1E82
:102FD00028E0C216D10431F70E948607B6CF202F11
:102FE000281B822FE8CFECEDF3E0818121E04381C3
:102FF0006281885F81CFECEDF3E0818121E0438144
:103000006281885079CFECEDF3E0628128E0620FB5
:1030100008F46FEF21E0438181816ECFECEDF3E0A6
:10302000628128E0621B08F460E021E04381818135
:1030300063CFECEDF3E0438128E0420F08F44FEF5B
:1030400021E06281818158CFECEDF3E0438128E0FB
:10305000421B08F440E021E0628181814DCF609104
:10306000DC036695669570E04BE050E088E091E007
:103070000E94F133892B19F481E08093DB030E94D5
:10308000920B9093B9028093B80208959091DC035B
:1030900090FF2CC0811559F18B3258F58F73880F32
:1030A000880F9091DC039370892B8093DC0361156A
:1030B00019F08CED93E0DFDE6091DC036695669598
:1030C00070E04BE050E088E091E00E94F133892B02
:1030D00091F01092DB0381E08093BB0220E04091ED
:1030E000DF036091DE038091DD0306CF089581E068
:1030F000D6CF8AE2D4CFB3DFEECF8091DC038695C2
:1031000086958F5F8B3208F081E061E0BFCF8091C0
:10311000DC03869586958A9509F48AE261E0B6CF4C
:10312000A8E0B0E0E6E9F8E10C9428337C01DC018A
:1031300014968C91811509F490C161E0C70189DB77
:103140008C01F7018581811521F18091D403909143
:10315000D5030097F1F008171907D9F0FC01FF27F4
:10316000887F9927892B09F072C074E0EE0FFF1F4A
:103170007A95E1F7EC5AFC4F858184608583118351
:103180000083CF01ACDA1092E70361E0C70161DB95
:103190008C01D70115968C91811509F4EEC0C801F8
:1031A00097578038910508F0DEC0003108F044C11F
:1031B00066E772E080E090E0ADDB81113DC1812CDB
:1031C000912C5401011146C004E09E012F5F3F4F36
:1031D0006901D601E02F1D92EA95E9F72401350136
:1031E000FFEF4F1A5F0A6F0A7F0AC501B40192DB35
:1031F0008983811509F420C1813009F0B1C0A5018E
:1032000094012E5F3F4F4F4F5F4F2D833E834F837F
:103210005887C301B2017EDB182F8A83811509F418
:103220000BC18FEF810F833080F56D817E818F819F
:10323000988570DB8B83811511F0C60195DB240125
:10324000350133E0430E511C611C711C1BC0E0E0D2
:10325000F0E092CFB7E78B16B2E09B06A104B10471
:1032600009F4EAC0C501B40155DBEFEF8E1A9E0ADE
:10327000AE0ABE0A8111EECF0150A4CF4D805E8010
:103280006F80788453014201A4CF8BEF810F83308C
:1032900090F52401350143E0440E511C611C711C62
:1032A0006D817E818F81988535DB8B83811551F30C
:1032B000C301B2012FDB8C83811108C024013501C9
:1032C00054E0450E511C611C711CDCCF8B819C812C
:1032D0008130AFEF9A0710F0982F8827163029F029
:1032E000173031F00E947526E9CF0E941126E6CFF3
:1032F0000E944326E3CF143009F0C0CF6D817E8158
:103300008F81988507DB182F24013501B4E04B0E1F
:10331000511C611C711CC501B4016D5F7F4F8F4F43
:103320009F4FF8DA111509F487C0811509F484C09C
:103330008150990B4FEF489F9001499F300D112408
:10334000E12FE150FF0B2E0F3F1F2150310908F4F0
:1033500099CF8FE99FE00197F1F700C00000F5CF0A
:10336000C60102DB8FCFF801F857E730F10508F00E
:10337000DBC0EC50FB4C0C940D336801A7E5DA1A66
:10338000C114B1E0DB0608F0CFC065E473E08C2D1A
:103390004DDC892B21F5C60154E0880F991F5A9501
:1033A000E1F7FC01EC5AFC4F2281213061F52091BC
:1033B000450330914603232B91F020914703309130
:1033C0004803232B61F02091490330914A03409137
:1033D0004B0350914C03242B352B232BE1F0023A65
:1033E000B2E51B0709F4ECC008F0BFC0C801905259
:1033F0008115904208F4D6C0013E110509F4E0C0E1
:10340000053E1105B5C0223051F720914903309196
:103410004A03232B21F3FC01E75AFC4F20812E7F26
:1034200020838C5A9C4F5BD9DACF83E00E942C0A10
:103430008FE493E00E94FA0E8091E8038770811573
:1034400061F0D70115968C91811539F080919F0418
:1034500082FF03C082E00E949D042896E0E10C9464
:10346000443380E0E3CF80914F03883088F0885068
:1034700080934F0391E0883008F490E080914F03EF
:1034800090FB80F980934F038FE493E00E94FA0E43
:1034900080914F038695869586950E94090ACCCF28
:1034A00090914F03892F869586958695983140F4A3
:1034B0008F5F880F880F880F9770892B80934F0339
:1034C00080914F038160DECF80914F0380FF09C060
:1034D0008E7F80934F038FE493E00E94FA0E80E08A
:1034E000DCCF816080934F03813071F689E0CACFD1
:1034F00080914F038695869586958F5F8F71843076
:1035000008F080E0880F880F880F90914F03977024
:10351000892BAECF80914F0381FF03C00E94160F0D
:103520008BCF0E94000F88CF0337ECE71E0709F00E
:1035300056CFD70115968C91811509F47DCF8091D6
:103540005003811511F0A6D877CF1092E5030E94A1
:10355000C6040E94920B88579C4E9093520380930E
:10356000510381E08093500367CF023B22E51207AD
:1035700009F03FC025EE30E02770332781E090E06E
:1035800001C0880F2A95EAF7209153033091500328
:103590003115F1F0F70135813115A9F0282B209371
:1035A00053034ACFD70116968C91803110F5812FA5
:1035B00099278F7199278230910511F04297D8CFC2
:1035C00021EE30E0D9CF809582238093530334CF0E
:1035D000322F3823311569F0982F909592239093CC
:1035E00053030E94BE04D70115968C91811509F4EE
:1035F00023CF80915003811509F4C4C0C090E50326
:10360000D090E4030E94920B88579C4E90935203F3
:1036100080935103F7018581811509F4B3C08D2D85
:103620008C298D7981117FC00115F0E51F07F8F411
:10363000011520E4120708F08EC0063E1105F1F1D5
:10364000C80190528115904208F08CC0D70116969F
:103650008C91803108F45FC0C80199271092E7036C
:103660008D329105A9F482E08093E7037FC0043B8B
:10367000B2E51B0719F108F041C00034F2E51F075D
:10368000B8F4011522E51207C8F41092E703C80147
:103690008E32910508F0BDC08832910508F064C0F3
:1036A0008E31910508F062C004974A97E0F23BC062
:1036B000C801805692458034910538F7F70195810D
:1036C000911509F4F5C41092D803980130572332AC
:1036D000310508F0D4C484E090E00E942F34909328
:1036E0009F0480939E04F801E150F047E232F10517
:1036F00008F0E3C0E550FB4C0C940D33003E32E57E
:10370000130720F4003C42E51407BECFC8018757D9
:103710009C470297D2CF812F8F71843179F2863105
:1037200049F41092E7030E944A13809153030E94C8
:10373000B80428C00E944A13809153030E94B80421
:10374000F801E851FC47E730F10508F0B7CFE35E38
:10375000FA4C0C940D33D70116968C91803108F0F9
:103760007BCFEECFC8017ACF8A97E9F680915303D9
:10377000811531F08091E70392E089278093E70378
:103780000E94520FC801975581159140C8F6580103
:10379000F8EFAF22BB24A114B10409F04DCEF8011B
:1037A000FF2734E0EE0FFF1F3A95E1F79F012C5AF7
:1037B0003C4F6901D70115968C91E75AFC4F9081D7
:1037C00080FB90F99083811559F10E94920B9093A0
:1037D000D7038093D603F60182818F5F8283809125
:1037E000E7039091E503892B83838091E40384832D
:1037F0004681578166857785C6010E94030BD601F5
:1038000015968C9181FF5801B092D503A092D403F4
:1038100055CF8C34910509F4A9CF8D329240A5CFB4
:10382000F9014485558566857785C9010E94030B9A
:10383000D60115968C9181FF41CFC6010E9453138A
:103840008091D4039091D5030817190709F036CF5A
:103850001092D5031092D40331CF06E221EE41EE4F
:103860006AE17CE7F701858108C007E225EE45EEB5
:103870006BE17CE7D70115968C9108DADDCD06E285
:1038800021EE40EE68E17CE7EDCF07E225EE44EE65
:1038900069E17CE7EFCF06E221EE42EE6CE17CE7E6
:1038A000E1CF07E225EE46EE6DE17CE7E3CF08E2EB
:1038B00021E045EE6EE17CE7D5CF80919E048160EA
:1038C00080939E0460919E0470919F0484E090E038
:1038D0000E945D340E94A10FAFCD80919F0488604B
:1038E00080939F04EFCF80919E048260E9CF809106
:1038F0009E048460E5CF80919E048860E1CF809132
:103900009F048160EDCF80919F048260E9CF809118
:103910009E048061D5CF80919E048062D1CF80913A
:103920009E048064CDCF0E94A10F80919E04806888
:10393000C7CF80919E048C60C3CF80919F04836029
:10394000CFCF80919E048E7FBBCF80919F04877FD5
:10395000C7CF80919E048D7FB3CF80919E048B7FD3
:10396000AFCF80919E04877FABCF80919F048E7FE5
:10397000B7CF80919F048D7FB3CF80919E048F7EBF
:103980009FCF80919E048F7D9BCF80919E048F7BE3
:1039900097CF0E94A10F80919E048F7791CF809145
:1039A0009E04837F8DCF80919F048C7F99CF8091DF
:1039B0009E04992782FF939590FB82F990FB83F9EF
:1039C0007FCF80919F04982F909590FB80F990FB7A
:1039D00081F986CF90919E04892F8F7B96FF80641A
:1039E0006FCF0E94A10F90919E04892F97FB87F9BA
:1039F000805866CF61E08EE090E00E94433462CF51
:103A000060E0F9CF90919E04892F8F7E94FF8061B2
:103A100057CF90919E04892F8E7F90FF816050CF69
:103A200090919F04892F877F93FF886059CF82727E
:103A3000F801E052F847EB30F10508F04CC0EC5DBE
:103A4000FA4C0C940D330737FCE71F0709F047C009
:103A500081E00E94FC0365C08091DC0380FF0BC005
:103A60008E7F8093DC038CED93E005DA1092DB030C
:103A70000E948607E1CC81608093DC0361E086953B
:103A8000869504DBD9CC811521F041DBD5CC81159D
:103A9000E1F333DBD1CC811521F0ADDACDCC81154A
:103AA000E1F3A1DAC9CC811521F0B8DAC5CC8115D2
:103AB000E1F3A9DAC1CC811521F0C6DABDCC8115BC
:103AC000E1F3B7DAB9CC811521F00CDAB5CC811568
:103AD000E1F3FED9B1CC07372CE71207F9F008372C
:103AE0003CE7130721F19801205E32452032310571
:103AF00018F5911138C00F7181E090E0AC0102C05F
:103B0000440F551F0A95E2F78A01642F83E090E085
:103B10000E944334802F0E94EC038ECC81E00E94EF
:103B2000F20343E062E081E00E94740485CC82E00D
:103B3000911509F48ECFF3CF9115A9F00A355CE702
:103B4000150709F476C008F04EC001309CE719074C
:103B500009F46DC00330ACE71A0709F462C001151F
:103B60001C4709F451C0F70187819085009709F43B
:103B700064C00E94C4058C01F701B580A680A294A0
:103B80002FE0A2228091E8038770811501F1CB2CF0
:103B9000B114F1F0812F807F803461F080E2800FDA
:103BA0008830A8F0812F807E803221F4023078F0B6
:103BB000A11469F080919F0482FF09C082E00E94F5
:103BC0009D048091E8038770CC24C3948111C12C9B
:103BD000E12FE295EF70103C08F0A1C0F0E0E15D4C
:103BE000FA4C0C940D330B35ECE71E0721F1809154
:103BF0009F04002482FF0394802D0C351C4709F09C
:103C0000B2CF0E94E30EAFCF0E94A10F2FEF34E39B
:103C10004CE0215030404040E1F700C000000E94DD
:103C20005D0E6FEF7FEF80E090E00E945D340E94B8
:103C3000C40F81E0E6CF80E0E4CF8581C080D180F1
:103C4000811569F0C6010E94FF13182F682FC60165
:103C50000E940A04B601812F0E94E4138ACFC60194
:103C60000E944004182FF6CFF12FFF70DF2E103185
:103C700018F0D29490EFD922B114A9F0D11459F0D0
:103C800080E2800F883010F0011107C08D2D0E9456
:103C9000B8040E94520F802F40C08091E7038D2905
:103CA0008093E703F6CF802F0E94E712D114B9F179
:103CB00080E2800F883010F0011104C08D2D0E9429
:103CC000BE0406C0D0948091E7038D218093E70362
:103CD0000E94520F24C0212F2F70D22E107F10323D
:103CE00019F0D29480EFD822011549F0013009F47F
:103CF00082C0B11409F48EC0A114A1F1CCCF80917F
:103D00009F0482FD2BC0B11419F1D11429F08D2D1F
:103D10000E94B8040E94520F80E00E949C12C114BD
:103D200009F4D8C08091E80380FDD4C0D70115966E
:103D30001C928695869586950E94F203C701F0D95C
:103D40008091E8038695869586950E94FC03C2C003
:103D500080E00E94E712D11411F3B0CFB11469F1E1
:103D6000A11004C08D2D0E942B13D9CF31E0A312D6
:103D700010C01091E4038D2D8123D81681F20E948A
:103D8000920B9093EC038093EB031D291093E403B3
:103D9000C6CF45E0A412C3CF8D2D0E942B138D2DCD
:103DA0000E94B20B8091E6039D2D9823D91609F449
:103DB000B6CF8D298093E603B2CFA11012C08D2D0E
:103DC0000E9431138D2D0E94B20B8091E6039D2D30
:103DD0009823911509F4A3CFD094D822D092E6036A
:103DE0009ECF51E0A5129BCF8091E5038D218115D7
:103DF00009F495CFE4CFB11429F086E0A81608F0B5
:103E00008ECFB0CF95E0A91608F089CF8D2D0E94F6
:103E1000311385CFA114D1F3093349F4AFEFB7EED5
:103E2000E3E0A150B040E040E1F700C00000802F87
:103E30000E94E71274CF812F869586958370811535
:103E400061F0813009F06BCFC8019370B11002C0EE
:103E500080E090E00E943F0B62CFC8019370B110E8
:103E600002C080E090E00E94170B59CF6B2D802F8D
:103E70000E94F00B54CF812F8370811138C0B11094
:103E800027C0402F429546954770440F440F802F1E
:103E90008F70042E01C0880F0A94EAF7202F20713A
:103EA00004FF07C02FE030E001C0220F4A95EAF777
:103EB00020951695169513701230A1F0133081F0ED
:103EC00030919C04113059F0822B83230E94EC0323
:103ED0000E94080B60E0C7010E942914BECA832B10
:103EE000822BF4CF822B90919C048927EFCFB114C1
:103EF00051F110FFEDCF402F429546954770440F8A
:103F0000440F802F8F70042E01C0880F0A94EAF7A7
:103F1000202F207104FF07C02FE030E001C0220FE6
:103F20004A95EAF72095169516951370123089F088
:103F3000133069F030919D04113041F0822B8323BE
:103F40000E94EF03C5CF823018F2D5CF832B822B8E
:103F5000F7CF822B90919D048927F2CF1F70B11467
:103F600039F0812F0E94F203802F0E942B13B0CFD3
:103F7000802F0E943113812F0E94FC03A9CF023FA2
:103F800071F170F4003FC9F0013F91F0B11409F4F0
:103F900065C0A11409F45FC0802F0E949C1298CFC5
:103FA000033F21F1043F91F780919F0482FD2AC0D5
:103FB000812F8F71B11401F316C0B11469F0F5E0CF
:103FC000AF1608F085CF1F7181E090E0012E01C08F
:103FD000880F0A94EAF7BECF26E0A216F2CF812F0F
:103FE0008F71B110C9CF0E94F20372CF80E0B1147B
:103FF00009F4A6CF1F7181E0012E01C0880F0A9439
:10400000EAF79ECFB114C1F08091E8038770843045
:1040100049F41092E8031092EA031092E903812F09
:104020008F71AACF35E063E0A31608F051CF812F3E
:104030008F710E949E0B4CCF45E0A41640F0109269
:10404000E8031092EA031092E90364E0F0CF81E004
:104050000E949D043DCF812F8F71C5CFA114F9F22D
:10406000093349F45FEF87EE93E051508040904070
:10407000E1F700C00000802F0E94E71229CF809155
:10408000E5030631FCE71F0709F0D1CC8A7A91E0FD
:10409000811101C090E09093D90365E3811101C0C3
:1040A00069E280EE91E00E94670B0E94520FC4C942
:1040B00006312CE7120709F0C6CC8091D90365E3DD
:1040C000811101C069E280EE91E00E94810BEDCF89
:1040D000A0E0B0E0EEE6F0E20C94313380913003E2
:1040E000803108F049C080912F03811509F444C044
:1040F000C091E10289E0D82E8091E0028C17E1F1B5
:10410000EC2EF12CDC9EE0011124FE01EE51FD4F5E
:1041100084818115B1F1918180912B03981331C075
:10412000908180912A0398132CC08581811129C028
:104130000281138180912C0390912D03081B190B90
:1041400060E08AE293E00E9429140E942B1608176F
:104150001907B8F4809130038F7080618093300329
:10416000C851DD4F88818F70806188838AE293E037
:104170000E9490180E949304CDB7DEB7E7E00C943C
:104180004D33E7012196C770B7CFAFE0B0E0EBEC5D
:10419000F0E20C9429338C0186E0F801DE011A96D6
:1041A00001900D928A95E1F7F801F580E4808AE2AA
:1041B000882E83E0982E80912E03811117C0E11480
:1041C00091F0F11409F480C1C8010E9458148115BE
:1041D00009F47AC189E0F801AAE2B3E001900D92F6
:1041E0008A95E1F775DFFF24F3946AC0A280B3805B
:1041F000D0902F0380912C0390912D033501681AE4
:10420000790AD11409F411C1C080518060E08AE2BA
:1042100093E00E9429140E942B166816790608F074
:10422000B6C0E11401F380912B03F8019181E09075
:104230003003F0E1EF1608F064C0981320C09091AD
:104240002A03F801808198131AC02091310330911C
:104250003203878190852817390789F4F1104BC004
:104260008E2D8F708061809330038AE293E00E94EC
:10427000901880913003F8018683F12C21C0F11051
:104280003AC040E0652D8C2D0E94180E40E0652D4F
:104290008C2D0E94180EF82E8111EFCF8A859B85F8
:1042A0000E944B14292F22952F70903470F49F7028
:1042B0002230A0F09115B1F0F8019681903190F480
:1042C0008F2D2F96EFE00C9445332A5F2F7022300C
:1042D00068F0C8010E949018FD2CF2CF911511F0E2
:1042E000811571F3805E883058F3F3CF803F40F33F
:1042F000815F8330F9CF80913003816080933003F8
:10430000BCCF98131EC090912A03F80180819813A6
:1043100018C020913103309132038781908528178E
:10432000390779F4F1100DC0E682C8010E94901897
:1043300089E0F801AAE2B3E001900D928A95E1F7D5
:1043400052CFC8010E945814811509F4BDC0F11460
:1043500009F4BAC080913003803208F43BCF8091D9
:104360002A0390912B039A838983BC82AB8280912C
:104370002E038D831E82EF82809131039091320350
:1043800099878887CE0101960E94901823CFD090FC
:104390003003F0E1DF1650F48AE293E00E949018B7
:1043A00089E0F40111928A95E9F767CFE11409F4E5
:1043B0001ACF90912B03F801818198131AC0909124
:1043C0002A038081981315C0209131033091320364
:1043D000878190852817390761F4F1100AC0D682C9
:1043E000C8010E94901889E0F40111928A95E9F7BA
:1043F000FACEC8010E945814811509F465C0F11461
:1044000009F462C080913003803208F4E3CE8091D9
:104410002A0390912B039A838983BC82AB8280917B
:104420002E038D831E82DF82A7CF60E08AE293E0B5
:104430000E9429140E942B166816790608F0B0CF46
:10444000E11409F4D0CEF11409F43EC090912B038D
:10445000F801818198132EC090912A0380819813CE
:1044600029C020913103309132038781908528172C
:10447000390701F580912C0390912D03A81AB90AF0
:10448000F8ECAF16B10408F053CF8091300380FDF3
:104490004FCF803108F44CCFF8018683982F907F5E
:1044A000903F09F442CF982F907F905F8F70892BB7
:1044B00086833BCFC8010E94581481118BCE809116
:1044C0003003816080933003C8010E9490188BCE26
:1044D000A2E1B0E0EEE6F2E20C9434330A871B87E7
:1044E0002C873D874E875F87688B798B8A8BCE01BF
:1044F0000A964BDE811128C02091E0023091E10242
:1045000089E0FE013A96DE01119601900D928A959E
:10451000E1F78E858115C1F0822F90E001968770BA
:10452000992738171906D9F099E0929FD0011124E4
:10453000AE51BD4FFE01319601900D929A95E1F773
:104540008093E0020E94930419E08091E10290912F
:10455000E002891312C06296E4E00C9450330E948A
:10456000A10F1092E0021092E10289E0EAE2F3E08A
:10457000DF011D928A95E9F7E7CF189FC00111244A
:104580008E519D4F02DE811531F38091E10290E062
:104590000196877099278093E102D7CFEF92FF921F
:1045A0000F931F93CF93DF9380919904E0910802BA
:1045B000CDE0811130C0CDB7DEB7E6E00C944E33CC
:1045C000D1E0DE0FD0930802EE2EF12CCE9FF00149
:1045D0001124EF5CFB4F84818115E1F08781908588
:1045E000892B21F481859285019651F400811181F6
:1045F000228133814481558166817781808568DF9E
:10460000CE9DF001CF9DF00D1124EF5CFB4F148285
:104610001092E703ED2F80919904E81788F2109229
:10462000990410920802C7CFA4E0B0E0EAE1F3E2F7
:104630000C94273320913004298397E0992E01E0D0
:1046400010E02DE0322E34E0532E882483948091A4
:104650002F049981891307C0A1DF0E94730A249651
:10466000E1E10C9443339981892F90E09C838B8303
:10467000FC01EE0FFF1FEB5DFB4F80819181989E47
:10468000D001999EB00D1124FD01E351FC4FFA8336
:10469000E983248121115BC060909904E1E3F4E097
:1046A00060E070E0712C661508F04FC0A384B484FC
:1046B000A981BA81CD90DC902FEF3FEF412C442DA2
:1046C00050E07601E40CF11CE40CF11CD701ED90F4
:1046D000FC90E114F10439F0AE14BF0409F0A90113
:1046E00043949A01ECCF2F3F3207D1F1D80102C099
:1046F000AA0FBB1F2A95E2F77A2A9801042C02C060
:10470000220F331F0A94E2F7A90141505109741690
:10471000150629F5369EF001379EF00D1124EF5C49
:10472000FB4F989ED001999EB00D1124A351BC4F10
:1047300012962D913C9113973087278354821082D3
:1047400011829287818715968C920E94840A8B81B0
:104750009C8101969A8389838370898378CF1482A0
:104760006F5F7F4F3D969FCF10929B0410929A04EB
:104770001092230180912F04809330040E94730AC9
:104780000DCFACE1B0E0E7ECF3E20C9426334B8BB9
:104790005C8B6D8B7E8B8F8BB92E988FA92E911190
:1047A0001092E703188A198A1A8A86E0FE01739626
:1047B000DE011A9601900D928A95E1F75F8880914B
:1047C0009F0482FF1FC00E94920B2091E903309149
:1047D000EA03821B930B8838934138F08091E803F9
:1047E00082FD03C082E00E949D040E94920B2091F2
:1047F000EB033091EC03821B930B8838934110F04C
:104800000E94C6045114D9F05E86BF8661E0CE01D5
:104810000A960E94291461E0CE010A960E9429148A
:1048200061E0CE010A960E9429144C0180356CE7A4
:10483000960791F4A11419F181E0809323015E861B
:10484000BF860A851B852C853D85452D5B2D688996
:1048500079898A893DDECDC081359C4721F4A11438
:1048600071F082DFECCF82E588168CE7980639F488
:10487000A11429F0809123018111F3CFDDCF4DEEFA
:10488000E42E43E0F42E412C612C712CD7016D9164
:104890007C91CC24CA94DD24DA9480E0282F30E087
:1048A000FB01E80FF11DE80FF11D40815181411519
:1048B000510539F08416950609F096018F5F69015C
:1048C000EDCF10E0BFEFCB16DB0609F44EC0F701C9
:1048D000448110912301411110E0D70115963C90BD
:1048E000159716969C911697A11409F405C11115F8
:1048F00009F402C1311017C021E030E00C2C01C0D6
:10490000220F0A94EAF7922B16969C9320912D047D
:1049100030912E042233310530F422E330E030931D
:104920002E0420932D04E1E0F0E002C0EE0FFF1F03
:104930008A95E2F7CF010197D70116962C91281797
:10494000190699F4C0909A04D0909B04C114D10424
:1049500009F453C00E94920B8C199D09C39708F467
:104960004CC081E0F701848311E0412ABFEF6B1A4C
:104970007B0AE7E0EE0EF11CF8E06F16710409F017
:1049800085CFA11409F417C1411409F414C10E9480
:10499000920B90939B0480939A04809199048830A1
:1049A00040F591E0980F9093990499E0FE013A96B2
:1049B000DE01119601900D929A95E1F75D82BE821B
:1049C0002DE0829FC00111248F5C9B4F29E0FE01E6
:1049D0003196DC0101900D922A95E1F72FEF3FEF20
:1049E000DC011A963C932E9319971C969C928E92FA
:1049F0001B976C96E2E10C94423320913004809135
:104A00002F04922FE0E0F0E001E0281709F448C0FD
:104A1000422F50E0FA01EE0FFF1FEB5DFB4F2080AD
:104A2000318037E0329DF001339DF00D1124E351C8
:104A3000FC4F608171817C8F6B8FB0E030E0A0E033
:104A4000EB8DFC8DEA0FF11DEA0FF11DC080D180C6
:104A5000C114D104E1F0F7010190F081E02DFA8F4B
:104A6000E98F30E007C0E1E0C616D70609F0E0E0C4
:104A7000BE2B3F5FE98DFA8DE30FF11DE30FF11DB2
:104A8000608171816115710571F7AF5FD9CFB11583
:104A900081F13A17C8F4E1E0D7011496EC93F701DD
:104AA00090933004EE15FF0509F45FCF90E0FC0110
:104AB000EE0FFF1FEB5DFB4F7182608201968370EA
:104AC000992780932F0451CF37E0329DF001339D19
:104AD000F00D1124E351FC4F0483EE15FF05F9F2AC
:104AE000291302C09F5F93709A012F5F3F4F23707D
:104AF0008CCFE0E0F0E0F8CF292F30E0311024C077
:104B000061E070E002C0660F771F8A95E2F7CB0183
:104B100001972817390791F010E0E1E0F0E002C0BA
:104B2000EE0FFF1FCA94E2F76F01C094D7011696EB
:104B30008C9116978C2116968C9317CF411569F39B
:104B4000C3010E94840AE8CFA9010C2C02C055952C
:104B500047950A94E2F7C901019782239323892B91
:104B600039F540FF25C0D70112968D919C91892B74
:104B7000D1F087E0FE013196DF011D928A95E9F7B9
:104B80000E94920B9C018B839C8384E08D83F701B0
:104B900092818381792F9887898709811A8144E0DE
:104BA0005E816F8195DCD70115961C92132DB5CFD0
:104BB000142F1170B2CF9091300480912F04981768
:104BC00031F032DDB1E04B1609F413CF38CEE6DC1C
:104BD00010929B0410929A040E94730AF3CFA6E0ED
:104BE000B0E0E5EFF5E20C9434330E94920B8C01B7
:104BF0008091D4029091D5028017910771F01982AB
:104C00001A820E94920BBC0149815A8180E090E097
:104C1000B8DD1093D5020093D4022696E4E00C94FC
:104C20005033A6E0B0E0E7E1F6E20C9434338C01B7
:104C30009093D1028093D002011580E21807B0F45E
:104C4000C801805E9109089728F067E373E10115B8
:104C5000110511F46BE273E1C8010E94C003802FBB
:104C60000E949C122696E4E00C94503380EF8983D6
:104C70008A830E94920B8160BC0149815A8181E044
:104C800091E07FDDEFCFA6E0B0E0E9E4F6E20C943E
:104C900034338C019093D1028093D002011580E2CD
:104CA0001807B0F4802F0E94E712C801805E9109B6
:104CB000089728F060E473E10115110511F461E330
:104CC00073E1C8010E94C0032696E4E00C945033BF
:104CD00080EF89838A830E94920B8160BC014981A5
:104CE0005A8181E090E04DDDEFCFCF93DF93D82F55
:104CF000C92F97DF8D2F9C2FC6DFDF91CF910895AD
:104D00000F931F93CF93DF938C01862F65E473E09D
:104D10000E941616892B91F4C0914503D091460349
:104D2000209761F0F8018281833039F4CE01DDDF14
:104D3000CE01DBDFCE01D9DF01C0E0F7DF91CF91FB
:104D40001F910F9108950F931F93CF93DF938C01C1
:104D5000EB0165E473E08C2F0E941616892B09F095
:104D600057C0FE01FF27D80112968C911297EF5879
:104D7000FD4F8130A9F415968C9182FD4EC080FFC5
:104D80004CC082E080838091470390914803009754
:104D9000B9F480914503909146030097C9F110C082
:104DA0008230A1F515968C9182FD26C080FD0AC047
:104DB00083E080838091490390914A030097F1F04A
:104DC00030DF26C084E0808380914B0390914C03B8
:104DD0000097B1F78091450390914603009701F148
:104DE00084DF8091470390914803009749F78091B1
:104DF000450390914603E4CF85E08083809145038D
:104E000090914603009721F070DFF1CF86E0808318
:104E1000DF91CF911F910F91089581E08083B9CFE9
:104E20008091470390914803B8CF0F931F93CF937E
:104E3000DF938C01EB0165E473E08C2F0E94161662
:104E4000892B71F4DD27CF58DD4F8881F80112825C
:104E500018828330E9F048F4813059F0823081F0D3
:104E6000DF91CF911F910F9108958430B1F085307B
:104E7000B9F78091450390914603009789F306C0E6
:104E80008091470390914803009799F3FCDEE8CFA7
:104E90008091490390914A03F7CF80914B03909101
:104EA0004C03009799F72091450330914603809178
:104EB00047039091480321153105F9F2009731F726
:104EC000C901E4CFA0E1B0E0E8E6F7E20C942833B2
:104ED000FE01319680E1DF011D928A95E9F708E233
:104EE00010E099E8A92EBB24B39427E7422E22E0D4
:104EF000522E612C712C4F0173016201B1E14B16EE
:104F00005104610471041CF080E1C82ED12CA6016B
:104F1000B501C4010E943434AC0CBD1C0D2C000C36
:104F2000EE08FF084C185D086E087F08015010401D
:104F300019F76096E0E10C9444336FEF85E290E05E
:104F40000E9443346FEF86E290E00E9443346FEF9B
:104F500087E290E00E94433460E088E290E00E94A3
:104F600043340E945C15AEDF6BE085E290E00E9466
:104F700043346BE486E290E00E94433462E687E2C9
:104F800090E00C9443348F929F92AF92BF92CF9255
:104F9000DF92EF92FF920F93CF93DF9388E090E040
:104FA0000E942A344B015C01CCEDD3E068839982E6
:104FB000AA82BB821C821D821E821F8283E290E035
:104FC0000E942234282F30E040E050E060E070E0A2
:104FD00080E090E000E20E945D33282939294A29C7
:104FE0005B29288339834A835B836C837D838E832B
:104FF0009F83DF91CF910F91FF90EF90DF90CF9043
:10500000BF90AF909F908F900895A6E0B0E0EBE046
:10501000F8E20C942B33FE01319686E0DF011D92FD
:105020008A95E9F787E6A82E81E0B82E0BE611E015
:10503000992493947E2E8F2EEE24E394F12C21E775
:10504000C22E21E0D22EF50181915F018F3F09F43C
:1050500046C0F894E82FE295EF70F0E021A18F7040
:10506000A70102C0440F551F8A95E2F7CA01922F8B
:10507000982B91A392A18095892382A3789400C054
:10508000ABE6B1E0672D782D492D40959D91FB0150
:105090008191BF019F3F09F447C0292F22952F70AE
:1050A000205E30E0F901208130E09F7002C035952C
:1050B00027959A95E2F720FD37C089299B01215059
:1050C0003109F9018083CA16DB0601F7F5018291E7
:1050D0008F3F11F00E94C206F0EAFA95F1F7990CA1
:1050E0000A151B0509F0AFCF46E050E0672D782D7B
:1050F00083EA92E00E94FE33892BC1F086E0E72D1F
:10510000F82DA3EAB2E001900D928A95E1F781E0D3
:105110008093EA010E94920B9093E9018093E80149
:105120002696EDE00C9447338423C8CF8091EA01A2
:105130008115B1F30091E8011091E9010E94920BF1
:10514000801B910B059760F346E050E063EA72E044
:1051500087EC92E00E94FE33892B49F086E0E3EA77
:10516000F2E0A7ECB2E001900D928A95E1F710927F
:10517000EA01D6CFCDB7DEB7AC970FB6F894DEBF55
:105180000FBECDBF85B7806885BF85B7806885BFF6
:1051900084B7877F84BF0FB6F894A895809160008C
:1051A000886180936000109260000FBE80E890E0FC
:1051B0000FB6F89480936100909361000FBE81E078
:1051C0008093160180EC96E09093DF018093DE01DE
:1051D0000E944E0A0E94D2150E94610D0E94BE0DCF
:1051E0008091E20084608093E20078948091CF0205
:1051F000811599F08091E9001091EC008F7017955E
:1052000011271795182B1092E9008091E80083FD73
:105210000E94D90F1F701093E90082E084BD93E0D3
:1052200095BD9AEF97BD80936E000E949B148111EB
:1052300001C083DE85EF0E94C20684EF0E94C20691
:1052400083E90E94C20682E90E94C2060BE611E0D1
:10525000D8018D918D018F3F11F00E94C206B1E0FF
:1052600001371B07A9F786E0E7ECF2E0DF01282F02
:105270001D922A95E9F7E3EAF2E0DF011D928A9593
:10528000E9F780E090E00E942F34833E9E4F21F4A6
:105290000E949B1481112FC063EE7EEF80E090E0AE
:1052A0000E945D3460E082E090E00E94433481E03F
:1052B00080939C0461E083E090E00E94433460E0CE
:1052C00074E184E090E00E945D341982CE01019681
:1052D0000E94FA0E0E945C1730DE40E050E0BA01F6
:1052E0008FE090E00E94553440E050E0BA0183E145
:1052F00090E00E94553482E090E00E942234809336
:10530000B10284E090E00E942F3490939F04809338
:105310009E047BDEEFEFF6E721E0E150F040204015
:10532000E1F700C0000071DE8091C70280FF08C075
:105330006FEF7FEF80E090E00E945D340E945D0E91
:1053400083E090E00E9422340E94EC03279A2F9879
:105350008AE08093800089E1809381008FEF9FEF46
:1053600090938700809386000E94941380914F034E
:1053700081FF0BC01092AB021092AA021092A902F8
:1053800080916F00816080936F000E9494138091E0
:10539000AC0281111EC08CED93E0F5DD8091DC0341
:1053A000843028F40E945C178CED93E0ECDD0E94C1
:1053B00071071092DB030E94660A8091DC0380FF74
:1053C00005C060E0869586950E94461881E080932E
:1053D000AC0287E191E09093D7028093D60280914E
:1053E000CF0210E4853009F490C00FDE02EB12E02A
:1053F00047ECE42E42E0F42ED701F80191918D9113
:1054000022E0E83BF20709F49EC09817B9F3D12CCB
:10541000D701CD907D01F80191908F019C1421F16D
:105420009C24B12CAA24A394892D8A218115A9F04A
:10543000B982DA820E94920B9C838B83F1E0FD8318
:1054400091E08C2D8A21811101C090E09E834981D9
:105450005A816B817C818D8194D9B394AA0C24E00C
:10546000B212E2CFF801C292D39436E0D312D0CF79
:105470000E94AB0C6BC08091CF02843009F43AC01B
:1054800080E00E942C0A1092DB038091AF02811110
:105490000EC031E03093AF028091DC03982F917001
:1054A0009093AE028E7F8093DC030E948607109259
:1054B000AD0288E190E00FB6F894A8958093600063
:1054C0000FBE1093600083B7817F846083BF83B772
:1054D000816083BF7894889583B78E7F83BF0FB632
:1054E000F894A89580916000886180936000109284
:1054F00060000FBE8ADDE7ECF2E0819181113EC6CB
:10550000ADECB2E0AE17BF07C1F78091CF02853096
:1055100009F4B1CF0E94A10F0E9494130E94080BBE
:105520001092AF028091AE02811551F08091DC03A0
:1055300081608093DC0360E0869586950E94461822
:105540000E942F1852CF981362CF49DBE090D4030A
:10555000F090D503E114F10439F1C090D603D09056
:10556000D7030E94920B8C010C191D09C7010E94E0
:105570002B1680179107C0F42091D4033091D503E6
:10558000C9019927287F3327232B09F0A0C134E0D4
:10559000880F991F3A95E1F78C5A9C4FDC011596BC
:1055A0002C9122FF0E946F1380912301811511F12C
:1055B00000919A0410919B0401151105D9F00E94E5
:1055C000920B801B910B20912D0430912E042817F3
:1055D000390780F49091300480912F04981709F4D2
:1055E00079C122D810922D0410922E0410929A04A0
:1055F00010929B0480915003811569F00E94920BD8
:105600002091510330915203821B930B8F3F9F4790
:1056100010F40E944A138091DB03811509F444C001
:105620008091DA03E091DC03E695E695E81BE093D0
:10563000BA02853109F4B9C108F064C1893009F4AE
:10564000A8C108F050C1823009F48DC1863009F438
:1056500095C100ED17E02BEDE22E26E0F22E8091B1
:10566000BB02811561F01092BB020E94920B9093D5
:10567000B9028093B8021092BC021092BD020E943F
:10568000920B2091B8023091B902821B930B8F3F8D
:105690009F4750F4200F311F3093B9022093B80276
:1056A00088EB92E0F701099586E0EFE3F3E0DE0195
:1056B000119601900D928A95E1F7B0904003D09039
:1056C0004103F0904203C0904303E09044031092E2
:1056D00041031092420310924303109244038F2D12
:1056E0008D29811509F441C00091C0021091C102B9
:1056F0000E94920B9C01201B310B90913D03911550
:1057000009F437C52531310580F19F3F19F09F5FBE
:1057100090933D03D11459F00E94BE0A91E01D14EC
:105720000CF09FEF899F802D112480934103F11489
:1057300059F00E94BE0A91E01F140CF09FEF899F60
:10574000802D11248093420380914103811569F0DB
:1057500010914203111549F00E94B00A8093410351
:10576000812F0E94B00A809342038C2D8E298115CF
:1057700009F441C00091BE021091BF020E94920B39
:105780009C01201B310B90913C03911509F4ECC452
:105790002135310580F19F3F19F09F5F90933C03C5
:1057A000C11459F00E94DE0A91E01C140CF09FEF26
:1057B000899F802D112480934303E11459F00E94A6
:1057C000DE0A91E01E140CF09FEF899F802D1124BA
:1057D0008093440380914303811569F01091440341
:1057E000111549F00E94B00A80934303812F0E9453
:1057F000B00A80934403809140038B1119C08091BB
:105800004103811511F08D1113C020914203211520
:1058100011F02F110DC090914403911511F09E11BC
:1058200007C030914303311103C0822B892B8111B2
:105830000E94C70B86E0FE013196AFE3B3E0019012
:105840000D928A95E1F70E94080B9091C202891788
:1058500021F08093C2020E94AB0C8091CF02843071
:1058600009F0BDCD83E08093E9008091E80082FFDC
:10587000B6CD8091E80090E085FF06C00E94300D13
:10588000811509F49DC091E08091E8008B778093A9
:10589000E800911509F4A3CD0091D2021091D30232
:1058A000E9810115110509F4A8C0EE3F09F0C8C04F
:1058B0008A81833020F08550833008F0C1C0EA81AE
:1058C000EE3008F0BDC0F0E0E55CFA4CA6C680E022
:1058D00090E064CE0E94CE2210929A0410929B0413
:1058E0000E94730A87CE8F3009F0B3CEE695F0E0C0
:1058F000E752FA4FE4910E2F10E0A1E3EA2EA8E060
:10590000FA2EADCE04EF11E067E5E62E69E0F62E43
:10591000843209F4A4CEA8F408E210E053EDE52E99
:1059200058E0F52E883109F49ACE833209F091CEF1
:10593000E4EDF5E005911591E8EBEE2EE7E0FE2EA3
:105940008ECE853209F085CE8E2F63E033D6E92FD7
:10595000F0E0EF52FA4FE4910E2F10E076EAE72ED6
:1059600076E1F72E7CCEF0E0EE51FA4FE4910E2F67
:1059700010E095EFE92E97E0F92E71CEF0E0E152BC
:10598000FA4FE4910E2F10E086EEE82E87E0F82E15
:1059900066CEE695F0E0E452FA4FE4910E2F10E067
:1059A000B8E0EB2EB8E0FB2E5ACEF0E0EA52FA4F08
:1059B000E4910E2F10E0F8E8EF2EF8E0FF2E4FCE26
:1059C00000E210E09E012F5F3F4F79018091E800D7
:1059D00085FD0AC08091E8008B778093E8000E94E3
:1059E000300D811599F34FCF8091F100D7018D9340
:1059F0007D010150104051F746CFE43148F4E115E4
:105A000051F0E150E33138F4F0E0E75BFA4C05C6C1
:105A1000EE3F09F454CF8FEF898312C01A8289E0D8
:105A20008B830EC08A81823081F08330B1F0813067
:105A300091F70E94AB0CF7D56B837C838D839E839B
:105A4000CE0101960E94800DCACC88E290E0FAD681
:105A50001B821C821D828E83F3CF8091CD02909198
:105A6000CE02892B69F386E0E7ECF2E0DE011396C3
:105A700001900D928A95E1F7E3CF8A81823059F641
:105A80006B817C818D819E81CED588E290E0FBD6B2
:105A9000D7CF4C816B818A810E94B61398278927C2
:105AA00098279E838D83CCCF2D813E81322723275B
:105AB00032274C816B818A810E942C0FC1CF0E94BA
:105AC0005C15BECF8A818930E9F08A3049F18A813C
:105AD000823809F449C068F58038A1F1813809F0AD
:105AE000AFCF60E08B810E9446189B818091DC03E0
:105AF000911131C08E7F8093DC031092DB030E94F2
:105B000086079ECF2B8130E0C901880F991F820F35
:105B1000931F6FEF70E05AD5862F0E942C0AD7CFC3
:105B20008B81811103C00E94160FD1CF0E94000FFC
:105B3000CECF833809F084CF20E04091DF036C8121
:105B40008B8106C020E04B816091DE038091DD03F4
:105B50000E947C1775CF81608093DC0360E086959E
:105B600086950E9446186CCF8B818093E00368CFA6
:105B70008A81893089F08A30C9F0823859F1D8F4A5
:105B8000803819F1813809F05BCF8091DC0380FF08
:105B90001FC08695869544CF80914F038695869544
:105BA0008695B5E58B9FC00111243ACF80914F03B4
:105BB0008695817035CF833809F042CF8091DD031F
:105BC0008B838091DE038C833BCF8091DF0328CFD2
:105BD00080E026CF8091E00323CF8FE493E00E9402
:105BE000FA0E0E9471078CED93E00E943B1728CFBC
:105BF00080E18A8325CF82E08A8387E711CF8C8179
:105C00008D3108F01DCF8A809B80982489249824A8
:105C1000A12CB12C8E010F5F1F4F7801E80EF11CF3
:105C2000E016F10609F40CCF80E0E7E78E16E2E01B
:105C30009E06A104B10420F4C40187579E4F02D6EA
:105C4000D80114968C930F5F1F4FBFEF8B1A9B0ADE
:105C5000AB0ABB0AE5CF8091CD029091CE02892B91
:105C600009F4EECE8C818D3108F0EACE882E912C8D
:105C7000A12CB12CCA80DB80DC24CD24DC24E12CD7
:105C8000F12C8E010F5F1F4F412C512C3201481413
:105C900059046A047B0408F0D3CEE7E7CE16E2E0AD
:105CA000DE06E104F10438F4D80114966C91C601C3
:105CB00087579E4FE8D5BFEF4B1A5B0A6B0A7B0AEA
:105CC000EFEFCE1ADE0AEE0AFE0A0F5F1F4FDFCF9C
:105CD000F9D8B6CE84E08DCF8C818D3108F0B0CE6E
:105CE000882E912CA12CB12CCA80DB80DC24CD2401
:105CF000DC24E12CF12C412C512C32018E010B5F64
:105D00001F4F481459046A047B0408F099CE80E0C0
:105D1000F0ECCF16D104E104F10418F4C601899621
:105D200091D5D8018D938D01BFEF4B1A5B0A6B0A99
:105D30007B0AEFEFCE1ADE0AEE0AFE0AE2CF2C81D2
:105D4000022F10E02D3108F07BCE8A819B819827AD
:105D5000892798272C01612C712C803C910508F033
:105D60006FCE822E912CA12CB12C40EC50E060E043
:105D700070E0441955096609770942175105610514
:105D8000710508F45DCE2091CD023091CE02232B17
:105D900009F03EC01C01F9E22F0E311C80FBEE24FD
:105DA000FF24E0F880FF0BC088964CD59D818927A1
:105DB0009827892781159C4711F48FEF8D83D50192
:105DC000C401840D951DA61DB71D80FF19C0680173
:105DD00031E0C31AD108CE0105968C0D9D1D9CA7FC
:105DE0008BA7C101800F911F2DD5ABA5BCA59C91A0
:105DF00081159C4721F48FEFEBA5FCA580838601DC
:105E0000FE013196EE0DFF1D2FEFE016F10638F082
:105E10008E010F5F1F4FC12CD12C760124C09481BD
:105E2000858181159C4711F42483258342E0E40E8B
:105E3000F11C3296EACF80EC4816510461047104DB
:105E400030F4D80114966C91C20189961CD5BFEF2D
:105E5000CB1ADB0AEB0AFB0AEFEF4E1A5E0A6E0A58
:105E60007E0A0F5F1F4FC814D904EA04FB0418F31D
:105E7000E7CD8091CD029091CE02892B09F4E0CD3F
:105E8000CE0101960E94800DFFEF21EE34E0F1502B
:105E900020403040E1F700C0000050CA88E0E4E252
:105EA000F1E0DE01919601900D928A95E1F7FE01F5
:105EB00032968FE1DF011D928A95E9F786E08983AA
:105EC00088E07F96DE011596D3CD88E2898381E054
:105ED0008A831B821C82B4CD8B819C81092E000C8D
:105EE000AA0BBB0B25E0880F991FAA1FBB1F2A9581
:105EF000D1F7AC01BD01405E5F4F6F4F7F4F481738
:105F000059076A077B0708F49BCD8832E1E09E07BA
:105F1000A105B10508F094CD4932F1E05F076105B4
:105F2000710520F048E251E060E070E0481B590B39
:105F3000BC016A517A4FCE0101964AD481CD4AE123
:105F400050E06FEF70E0CE01079665D48091CD02EE
:105F500089830A831B821C821D8283E07CCD81E0C1
:105F600090E09093D3028093D20282E390E09093EA
:105F7000C6028093C5020E94920B9093C402809344
:105F8000C3025ECD0115110571F1D090C702E090FA
:105F9000C302F090C4020E94920B8E199F098536AD
:105FA000910540F1D3FE26C0D0FE24C00E94920B82
:105FB0009093C4028093C3028091C5029091C6025F
:105FC00001979093C6028093C502892B61F41092C9
:105FD000D3021092D20281E090E09093CE0280939F
:105FE000CD0200E010E08091CD0289830A83809188
:105FF000C50216CD82E390E09093C6028093C5025D
:10600000F2CF1092CE021092CD021ACD40E250E0B3
:106010006FEF70E0CE010196FED312CD8B818230FE
:1060200009F450C078F4811136C0FE0133968DE139
:10603000DF011D928A95E9F788E089838A8381E0F0
:1060400088A3FECC833009F472C0843009F0F8CC08
:106050001C818AE0FE013596DE01919601900D9239
:106060008A95E1F789A59AA50E94410A9AA789A76E
:106070008FEF183060F4FAE01F9FB0011124675CC5
:106080007E4F4AE050E0CE0181961BD480E08983A8
:106090000E94D215D5CC8C819AE0F92E8E010F5D2D
:1060A0001F4FF8012F2D11922A95E9F7B8010E9490
:1060B00016168983F801DE01129601900D92FA946A
:1060C000E1F7BECC1C818AE0FE013596DE01919697
:1060D00001900D928A95E1F789A19AA10E94410A47
:1060E0009AA389A38BA19CA10E94410A9CA38BA384
:1060F0008DA19EA10E94410A9EA38DA38FA198A568
:106100000E94410A98A78FA38FEF183060F43AE0FD
:10611000139FB001112467517F4F4AE050E0CE0138
:106120008196CFD380E089830E944E0A89CC2C814E
:106130006AE0CE018196DC01E62F1D92EA95E9F72F
:10614000283080F4629FB0011124675C7E4F4AE0E2
:1061500050E068D380E089838AE0FE01B196DE01D9
:10616000129686CC8FEFF7CF2B30310508F015CB88
:1061700042CB2B30310508F0CACAF7CA8091B00271
:10618000811509F4C2C9B0E1B9BDE2E1E9BD09B4C4
:1061900000FEFDCF8091D8008F7D8093D800809144
:1061A000E00082608093E0008091E00081FDFCCF00
:1061B0000E94A10FAAC91F920F920FB60F9211242D
:1061C0002F933F934F935F936F937F938F939F93FF
:1061D000AF93BF93EF93FF93809104018230A1F0BE
:1061E0008F5F80930401FF91EF91BF91AF919F91D9
:1061F0008F917F916F915F914F913F912F910F9070
:106200000FBE0F901F90189581E08093040180913C
:10621000AA029091AB02019660ED72E0D7D1909303
:10622000AB028093AA0265E070E0D0D167FD6FE712
:106230008091A902823069F5603429F480916F0061
:106240008E7F80936F00E62FF0E0E45BFC4F24919B
:10625000A0918600B091870030E098D32FEF30E016
:1062600040E050E071D3C90163E070E0AFD18091AC
:106270004F03869586958695282F269FC001279FD8
:10628000900D11240E948D0990938D0080938C00B5
:10629000AACF8130C1F66F37D0CF1F921FB61F92A1
:1062A00011248F939F93AF93BF938091AD0281117F
:1062B00013C08091000290910102A0910202B0915E
:1062C00003024196A11DB11D80930002909301022B
:1062D000A0930202B0930302BF91AF919F918F915F
:1062E0001F901FBE1F90189578941F921FB61F9283
:1062F00011248F939F93AF93BF938091000290914D
:106300000102A0910202B09103020196A11DB11DEC
:106310008093000290930102A0930202B0930302C3
:10632000BF91AF919F918F911F901FBE1F901895A5
:106330001F920F920FB60F9211242F933F934F93FA
:106340005F936F937F938F939F93AF93BF93EF93DD
:10635000FF938091E10082FF09C08091E20082FFFB
:1063600005C08091E1008B7F8093E1008091DA008D
:1063700080FF24C08091D80080FF20C08091DA0087
:106380008E7F8093DA008091D90080FFA9C080E1E0
:1063900089BD82E189BD09B400FEFDCF81E0809313
:1063A000CF028091EF01811109C00E94610D0E940E
:1063B000BE0D8091E20084608093E2008091E10054
:1063C00080FF1AC08091E20080FF16C08091E20039
:1063D0008E7F8093E2008091E20080618093E200F2
:1063E0008091D80080628093D80019BC85E08093AA
:1063F000CF0283E0809316018091E10084FF2FC0DB
:106400008091E20084FF2BC080E189BD82E189BDDB
:1064100009B400FEFDCF8091D8008F7D8093D80015
:106420008091E1008F7E8093E1008091E2008F7E79
:106430008093E2008091E20081608093E20080918D
:10644000EE01811509F452C084E08093CF0280915F
:10645000CF02843009F052C082E08093160180910F
:10646000E10083FF2CC08091E20083FF28C080916F
:10647000E100877F8093E10082E08093CF02109259
:10648000EE018091E1008E7F8093E1008091E20037
:106490008E7F8093E2008091E20080618093E20031
:1064A00042E060E080E00E948E0D8091F000886004
:1064B0008093F00081E08093160180931501FF9195
:1064C000EF91BF91AF919F918F917F916F915F916C
:1064D0004F913F912F910F900FBE0F901F901895E5
:1064E00019BC1092CF021092EF0168CF8091E300A7
:1064F00087FF02C083E0A9CF81E0A7CF81E0ADCFC5
:106500001F920F920FB60F921124EF92FF920F93EA
:106510001F932F933F934F935F936F937F938F932B
:106520009F93AF93BF93CF93EF93FF9309EE10E048
:10653000F8018081C091EC008F70C795CC27C7957A
:10654000C82B108280EFE82EF12CF7018081877F25
:10655000808378940E94D90FF8011082F70180811E
:1065600088608083CF70F801C083FF91EF91CF9155
:10657000BF91AF919F918F917F916F915F914F915B
:106580003F912F911F910F91FF90EF900F900FBEB1
:106590000F901F901895DB018F939F93C5D1BF91EA
:1065A000AF91A29F800D911DA39F900DB29F900D62
:1065B00011240895992778E0880F991F961708F0FD
:1065C000961B881F7A95C9F780950895AA1BBB1B57
:1065D00051E107C0AA1FBB1FA617B70710F0A61BE3
:1065E000B70B881F991F5A95A9F780959095BC0104
:1065F000CD01089597FB072E16F4009406D077FD81
:1066000008D0E4DF07FC05D03EF4909581959F4FBC
:106610000895709561957F4F0895EE0FFF1F0590C7
:10662000F491E02D09946927962769277827872711
:1066300078270895ABD1332312F48A1B9B0B01C03A
:10664000A5D1B7FF0895821B930B08952F923F9217
:106650004F925F926F927F928F929F92AF92BF9272
:10666000CF92DF92EF92FF920F931F93CF93DF931E
:10667000CDB7DEB7CA1BDB0B0FB6F894DEBF0FBE7B
:10668000CDBF09942A88398848885F846E847D84C8
:106690008C849B84AA84B984C884DF80EE80FD80CA
:1066A0000C811B81AA81B981CE0FD11D0FB6F89440
:1066B000DEBF0FBECDBFED010895002E083090F073
:1066C000982F872F762F652F542F432F322F222775
:1066D0000850F4CF220F331F441F551F661F771F2A
:1066E000881F991F0A95B2F7002D089597FD109401
:1066F000002E083098F00850232F342F452F562FA6
:10670000672F782F892F912DF4CF15949795879522
:106710007795679557954795379527950A95AAF7E1
:106720001124002D08958F929F92AF92BF92CF9225
:10673000DF92EF92FF92CF93DF93EC016881798132
:106740008A819B81611571058105910521F464E2BF
:1067500079ED8BE597E02DE133EF41E050E0C8D0D3
:1067600049015A019B01AC01A7EAB1E4DDD06B01FC
:106770007C01ACEEB4EFA5019401E2D0DC01CB01C9
:106780008C0D9D1DAE1DBF1DB7FF03C00197A10954
:10679000B04888839983AA83BB839F77DF91CF9189
:1067A000FF90EF90DF90CF90BF90AF909F908F9031
:1067B0000895B9CF80E091E0B6CFA0E0B0E080933B
:1067C000000190930101A0930201B0930301089589
:1067D000FB01DC0102C005900D9241505040D8F7FA
:1067E0000895FC014150504030F001900616D1F759
:1067F0003197CF010895882799270895FB01DC017F
:1068000004C08D910190801921F441505040C8F787
:10681000881B990B0895DC0101C06D9341505040D5
:10682000E0F70895DC01CB01FC01F999FECF06C029
:10683000F2BDE1BDF89A319600B40D92415050403E
:10684000B8F70895F999FECF92BD81BDF89A9927BE
:1068500080B50895A6E1B0E044E050E0E5CFA8E1BE
:10686000B0E042E050E0E0CFDC01A40FB51F4150A2
:10687000504040F0CB01840F951F2E9105D0415020
:106880005040D8F70895262FF999FECF92BD81BDCB
:10689000F89A019700B4021639F01FBA20BD0FB65E
:1068A000F894FA9AF99A0FBE08950396272FECDF11
:1068B000EADF252FE9DF242FE7CF0196272FE4DF3A
:1068C000E2CFDC01CB0102C02D9105D041505040F8
:1068D000D8F70895262FF999FECF1FBA92BD81BD32
:1068E00020BD0FB6F894FA9AF99A0FBE0196089552
:1068F000052E97FB16F400940FD057FD05D024D039
:1069000007FC02D046F408C050954095309521957B
:106910003F4F4F4F5F4F08959095809570956195CB
:106920007F4F8F4F9F4F089531D0A59F900DB49FFB
:10693000900DA49F800D911D11240895B7FFF4CFF1
:10694000F3DF821B930B0895A1E21A2EAA1BBB1B37
:10695000FD010DC0AA1FBB1FEE1FFF1FA217B3072B
:10696000E407F50720F0A21BB30BE40BF50B661F41
:10697000771F881F991F1A9469F760957095809505
:1069800090959B01AC01BD01CF010895A29FB0017C
:10699000B39FC001A39F700D811D1124911DB29F53
:1069A000700D811D1124911D0895F894FFCFFC0BEB
:1069B000010C030C080C180C180C180C180C180CF3
:1069C000180C180C180C0A0C0E0C110C160C260CBA
:1069D0002C0C300CB610DC10E210DC10E21034117C
:1069E0005511E2105B126812151A311A641A331A23
:1069F000501A781A8A1AA11C091DA91C731C771C2D
:106A0000AD1C7B1CB11CBD1C871C021D8B1CC11C3A
:106A10008F1CC51CEA1C931CC91CF11C991CCF1CA3
:106A2000D71C7F1CB51C831CB91C9D1CD31CE11CEE
:106A3000FA1C001D6D1CA51C101D3F1C451C2D1CA7
:106A4000351C4B1C511C571C2C1D431D471D4B1D39
:106A50004F1D531D571D5B1D5F1D631D671D341E9C
:106A6000341E6B1E6B1E1B1F361F8F1E8F1E3B1F7F
:106A7000AE1FBF1FBF1F4E2F652F6C2F202D202D47
:106A80009F2FAF2FC22F01300630202D202D202D1B
:106A90000E300E2D122D3D2D492D542D5F2D622DC2
:106AA000B82DED2D0B2D392FF82DFB2DFF2D2B2E75
:086AB000682E6A2E6C2E9F2E49
:106AB800010000000101010201191A1B1C1D1E1F03
:106AC800202122000001008F0BC30EB70CD90EDE67
:106AD8000EBA0E01FFF4B0ECBEE1355C0044227B37
:106AE80049012701AC004F02680288020001020236
:106AF80002020606060909090909090F0F0F0F0FF7
:106B08000F151515181919191919191919191923FA
:106B180024252525252525F5F493923336323197FA
:106B280034E200E900EA00B500B600B700CD008302
:106B380001CC008A0192019401210223022402253A
:106B480002260227022A02B300B4006F0070009FD9
:106B580001CB019F02A002E200E900EA00B500B6FD
:106B680000B700CD008301CC008A01920194012175
:106B780002230224022502260227022A02B300B4B5
:0E6B8800006F0070009F01CB019F02A0020071
:00000001FF
